:100000000C94DF050C94FC050C94FC050C94153045
:100010000C94FC050C94FC050C94FC050C94FC055C
:100020000C94FC050C94FC050C946C250C94A824F1
:100030000C94EA1E0C94FC050C94FC050C94FC0535
:100040000C94FC050C94FC050C94FC050C94FC052C
:100050000C94FC050C949D1E0C94FC050C94FC0562
:100060000C94FC050C94FC050C94FC050C94FC050C
:100070000C94FC050C94FC050C94FC050C94FC05FC
:100080000C94FC050C94FC050C94FC050C94FC05EC
:100090000C94FC050C94FC050C94FC050C94FC05DC
:1000A0000C94FC050C94FC050C94FC054F0A4F0ABB
:1000B000810A810AF30A0F0BA60CA60C1A0BF80B87
:1000C000090C090C26113611291136112C11361183
:1000D000361136112F1136112F1136112F113611FD
:1000E0002F11C122E8228024E822802430235323C8
:1000F00080244224552400DA0281FFD9F1DB20A4B8
:10010000A62EAF00A0C000A1C800AED580A81FD306
:1001100000408D1420001E0F0500047F3F1F643235
:1001200014643214783C1E1E140A0541646A757307
:1001300074005261697365004C6F776572004465A5
:100140006661756C74004C617965723A200080813B
:1001500082838485868788898A8B8C8D8E8F909107
:10016000929394A0A1A2A3A4A5A6A7A8A9AAABAC68
:10017000ADAEAFB0B1B2B3B4C0C1C2C3C4C5C6C7DF
:10018000C8C9CACBCCCDCECFD0D1D2D3D4002223B4
:10019000252628292A2C2D2F3032333536383A3B64
:1001A0003D3E4042434547494A4C4E5051535557B6
:1001B000595A5C5E6062646668696B6D6F717375D5
:1001C00077797B7D7F81838587898A8C8E909294D5
:1001D00096989A9C9E9FA1A3A5A7A8AAACAEAFB1E2
:1001E000B3B4B6B8B9BBBCBEBFC1C2C3C5C6C7C92C
:1001F000CACBCCCDCED0D1D2D2D3D4D5D6D7D7D8E6
:10020000D9D9DADADBDBDBDCDCDCDCDCDDDDDDDD37
:10021000DCDCDCDCDCDBDBDBDADAD9D9D8D7D7D63F
:10022000D5D4D3D2D2D1D0CECDCCCBCAC9C7C6C5F6
:10023000C3C2C1BFBEBCBBB9B8B6B4B3B1AFAEAC3C
:10024000AAA8A7A5A3A19F9E9C9A98969492908EE7
:100250008C8A89878583817F7D7B79777573716FC0
:100260006D6B6968666462605E5C5A59575553519C
:10027000504E4C4A4947454342403E3D3B3A383652
:10028000353332302F2D2C2A29282625232200AF62
:1002900000AE05010902A10185020901A1000509BD
:1002A000190129081500250195087501810205012C
:1002B000093009311581257F9502750881060938B5
:1002C0001581257F950175088106050C0A380215F0
:1002D00081257F950175088106C0C005010980A1AF
:1002E00001850319012AB700150126B7009501758C
:1002F000108100C0050C0901A101850419012AA083
:1003000002150126A002950175108100C0050109A2
:1003100006A1018506050719E029E71500250195C5
:1003200008750181020507190029EF1500250195BF
:10033000F0750181020508190129059505750191DE
:1003400002950175039101C005010906A101050788
:1003500019E029E71500250195087501810295012D
:10036000750881010507190029FF150026FF009572
:100370000675088100050819012905950575019183
:1003800002950175039101C009023B00020100A022
:10039000FA09040000010301010009211101000113
:1003A0002240000705810308000109040100010340
:1003B00000000009211101000122B6000705820397
:1003C0002000011201000200000008534601000154
:1003D00000010200010C0343006F0072006E006513
:1003E000000000100366006F006F0073007400616E
:1003F000006E000000040309040000000000003E3D
:100400005B4F5B3E003E6B4F6B3E001C3E7C3E1CD8
:1004100000183C7E3C18001C577D571C001C5E7F5A
:100420005E1C0000183C180000FFE7C3E7FF000057
:100430001824180000FFE7DBE7FF0030483A060EFB
:1004400000262979292600407F05050700407F0501
:10045000253F005A3CE73C5A007F3E1C1C08000820
:100460001C1C3E7F0014227F2214005F5F005F5F30
:100470000006097F017F00006689956A0060606060
:1004800060600094A2FFA2940008047E040800109B
:10049000207E20100008082A1C0800081C2A0808D2
:1004A000001E10101010000C1E0C1E0C0030383EE8
:1004B000383000060E3E0E0600000000000000006E
:1004C000005F000000000700070000147F147F1485
:1004D00000242A7F2A12002313086462003649563A
:1004E000205000000807030000001C22410000000B
:1004F00041221C00002A1C7F1C2A0008083E080814
:100500000000807030000008080808080000006043
:100510006000002010080402003E5149453E0000E2
:10052000427F4000007249494946002141494D330C
:10053000001814127F10002745454539003C4A49F0
:100540004931004121110907003649494936004621
:100550004949291E0000001400000000403400003A
:100560000000081422410014141414140000412245
:100570001408000201590906003E415D594E007CF5
:100580001211127C007F49494936003E4141412207
:10059000007F4141413E007F49494941007F0909AF
:1005A0000901003E41415173007F0808087F0000A7
:1005B000417F4100002040413F01007F081422415B
:1005C000007F40404040007F021C027F007F040803
:1005D000107F003E4141413E007F09090906003E6F
:1005E0004151215E007F09192946002649494932B7
:1005F0000003017F0103003F4040403F001F2040B7
:10060000201F003F4038403F00631408146300037C
:1006100004780403006159494D4300007F41414182
:1006200000020408102000004141417F0004020143
:100630000204004040404040000003070800002042
:1006400054547840007F28444438003844444428B7
:1006500000384444287F0038545454180000087E61
:100660000902001824241C78007F08040478000084
:10067000447D4000002040403D00007F10284400A1
:100680000000417F4000007C04780478007C08046E
:100690000478003844444438007C18242418001896
:1006A0002424187C007C0804040800485454542472
:1006B0000004043F4424003C4040207C001C2040B7
:1006C000201C003C4030403C004428102844004C92
:1006D0009090907C004464544C44000008364100E3
:1006E000000000770000000041360800000201020F
:1006F0000402003C2623263C00000000000000000D
:10070000000000000000000000C0E0F0F8F8180051
:10071000C0F0FCFEFFFFFFFFFFFFFF7E00000000B8
:10072000000000000080C0E0E0E0E0E0E0E0E0C0C9
:10073000800000000080C0E0E0E0E0E0E0E0E0C039
:1007400080000000E0E0C0C0E0E0E0E00000E0E0A9
:10075000C0C0E0E0E0E0E0C0800000000080C0E059
:10076000E0E0E0E0E0E0E0C0800000000000000029
:1007700000000000000000E0F0F0F0E0ECEEF7F325
:100780007020007C7C7C7E007E7E7E7F7F7F0000F0
:1007900080C0E07E5B4F5BFEC00000C000DCD7DEA7
:1007A000DEDED7DC00C0000000000000000000001A
:1007B0000000000000000000000000000000000039
:1007C0000000F8FCFEFFE000FFFFFFFFFFFF80FFDF
:1007D000FFFFFFFFFFFFFFFF1F07010000000000FA
:1007E00000000000FFFFFF8100000000000081C347
:1007F000C3C30000FFFFFF8100000000000081FF75
:10080000FFFF0000FFFFFF01000000000000FFFFEE
:10081000FF010000000001FFFFFF0000FFFFFF9D40
:100820001C1C1C1C1C1C9DDFDFDF000000000000E6
:10083000000000000000000F1F3F7F7F7F7F7F3F91
:100840001E0C001F1F1F3F003F3F3F7F7F7F003078
:100850007B7F7830202030787F3B0003000F7F0FB4
:100860000F0F7F0F000300000000000000000000D9
:100870000000000000000000000000000000000078
:100880000000030F1F3F3F3F3F1F1F3F3F7F7F7F02
:100890003F3F1F3F7F7F7F7F7C7878381C0F0000B1
:1008A0000000000000010307070707070707070309
:1008B00001000000000103070707070707070703F8
:1008C0000100000007070700000000000000070704
:1008D00007000000000000070707000000010307F1
:1008E00007070707070707030100000000000000D3
:1008F00000000000000000000000000000000000F8
:1009000000000000000000000000000000000000E7
:1009100000000000000000000000000000000000D7
:1009200000000000000000000000000000000000C7
:100930000000000000000000002B0014001A000856
:100940000015001700E00004001600070009000A67
:1009500000E1001D001B000600190005000000005A
:10096000000000E30001512C002A00130012000CCB
:100970000018001C00340033000F000E000D000BA7
:100980000029003800370036001000110000000078
:10099000000000E600025128002B001E001F00206E
:1009A0000021002200E00000000000000000000024
:1009B00000E1000000000000000000000000000056
:1009C000000000E30001002C002A0027002600257B
:1009D0000024002300000000004F0052005100508E
:1009E0000000000000000000000000000000000007
:1009F000000000E600035128002B001E021F022009
:100A00000221022202E000000000000000000000BD
:100A100000E10000000000000000000000000000F5
:100A2000000000E30003512C002A002702260225C3
:100A300002240223023500310030002F002E002D49
:100A4000003502310230022F022E022D020000007A
:100A5000000000E60001002800005C00000000002B
:100A60000000000000C35CC65CC85CCA5C000000FB
:100A700000C45CC75CC95CCB5C00000000000000E7
:100A8000000000E30001002C000000000000000056
:100A90000000000000000000000000000000000056
:100AA0000000000000000000000000000000000046
:100AB000000000E600010028000001010101010121
:100AC0000101010202020202020202020303030305
:100AD00003030303040404040404040505050505D5
:100AE0000606060606070707070708080808090993
:100AF00009090A0A0A0B0B0B0C0C0C0D0D0D0E0E3E
:100B00000E0F0F0F101011111112121313141415D0
:100B10001516161717181819191A1A1B1B1C1D1D44
:100B20001E1E1F202021222223242425262627289A
:100B300029292A2B2C2D2D2E2F30313232333435CA
:100B4000363738393A3B3C3D3E3F404142434445CD
:100B5000464748494A4C4D4E4F50515354555658AC
:100B6000595A5B5D5E5F616264656668696B6C6D56
:100B70006F7072737577787A7B7D7E8082838587CC
:100B8000888A8C8E8F91939596989A9C9EA0A2A30A
:100B9000A5A7A9ABADAFB1B3B5B7BABCBEC0C2C40F
:100BA000C6C9CBCDCFD1D4D6D8DBDDDFE2E4E7E9CF
:100BB000EBEEF0F3F5F8FAFDFFFFAA7F55401124A4
:100BC0001FBECFEFDAE0DEBFCDBF12E0A0E0B1E0A4
:100BD000E4E7FBE602C005900D92AA30B107D9F711
:100BE00027E0AAE0B2E001C01D92AD35B207E1F7FF
:100BF0000E94EA0D0C94B8350C940000882321F073
:100C00000E9449260C9450260895882339F090912B
:100C10004E07892B80934E070C9450260895882305
:100C200079F19CEF980F913A30F4682F86EB96E0BB
:100C30000E94131F0DC090E2980F983058F48770EF
:100C400091E001C0990F8A95EAF7892F0E94492601
:100C50000C9450269BE5980F933020F480E090E0B0
:100C60000C94861F98E5980F973120F480E090E06F
:100C70000C94701F8D3E20F00E94D22C0C94E62D17
:100C80000895CF93882309F472C0C82F8CEF8C0F7E
:100C9000813AC0F580914B018823E1F0809177047F
:100CA00087FF18C0EC2FE695E695E695F0E0EA544C
:100CB000F94F8281282F30E04C2F477081E090E07F
:100CC00002C0880F991F4A95E2F782239323892B4C
:100CD00061F412C0E8EBF6E08EEB96E02191C217CA
:100CE00021F08E179F07D1F707C06C2F86EB96E097
:100CF0000E94131F0E9450266C2F86EB96E00E94E4
:100D00003B1F10C080E28C0F883078F4C77081E000
:100D100090E001C0880FCA95EAF790914E07892BA1
:100D200080934E07CF910C945026EBE5EC0FE33007
:100D300040F4F0E0E555FE4F808190E0CF910C94B7
:100D4000861FE8E5EC0FE73150F4F0E0EE0FFF1FEF
:100D5000E255FE4F80819181CF910C94701FCD3E62
:100D600030F08C2F0E948B2DCF910C94E62DCF91DB
:100D700008951F93CF93DF93CDB7DEB767970FB674
:100D8000F894DEBF0FBECDBF4B8B5C8B6D8B7E8B23
:100D90008F8B611110924D0786E09E01235F3F4FBC
:100DA000D901E82F1D92EA95E9F795E0FE017396C7
:100DB000D90101900D929A95E1F79C894E895F893E
:100DC0007B897D879E876F87598B488BF901DE0170
:100DD000179601900D928A95E1F7CE0107960E9431
:100DE000CB2781113EC086E0FE013796DE011196C9
:100DF00001900D928A95E1F7FF81E8856A857B85F0
:100E00006115710531F0EF3F31F481E0FF3F19F4D6
:100E100003C081E001C080E080FD23C02091FA067C
:100E200030E0C90101968770992740912B0750E067
:100E30008417950779F1F983EA837D836C8396E0C3
:100E4000929FD001939FB00D1124A550B94FFE0180
:100E5000319601900D929A95E1F78093FA060E94DF
:100E6000C02616E080912B079091FA068917F9F0B9
:100E7000189FC00111248550994F0E94CB278823C9
:100E8000B1F080912B0790E00196877099278093AD
:100E90002B07E8CF0E94592A1092FA0610922B07CE
:100EA000E4EFF6E086E0DF011D928A95E9F76796A8
:100EB0000FB6F894DEBF0FBECDBFDF91CF911F916B
:100EC00008958F929F92AF92BF92CF92DF92EF924E
:100ED000FF920F931F93CF93DF93CDB7DEB72A977F
:100EE0000FB6F894DEBF0FBECDBFFC010081D180EC
:100EF00083819481892B39F01FEFD11206C091E0D4
:100F00000F3F19F403C091E001C090E090FD4FC67F
:100F10007F0185E0DE01169601900D928A95E1F73A
:100F2000F70122818E819F81222349F00E9436277A
:100F3000182F682F8E819F810E94992903C00E94DB
:100F40006C29182F20E3129FF001112436E0D39E64
:100F5000E00DF11D1124E00FF11DEE0FFF1FE75C06
:100F6000F64F05911491F70182818823A1F1C80100
:100F700090568115F0E29F0720F0905E8115904118
:100F800018F4C801992701C0C8018C33910528F4D1
:100F9000FC01E35AFE4F208101C020E21F922F93F3
:100FA0009F938F93F70180811F928F9381811F926E
:100FB0008F938CE491E09F938F931F9288E18F939E
:100FC00084E392E09F938F930E94C0320FB6F8940F
:100FD000DEBF0FBECDBF043F3CE5130759F190F4CF
:100FE000093D9CE51907E9F00A3DECE51E07A1F172
:100FF000083DFCE51F07B1F506E221EE41EE68ED84
:101000007CE514C0063F2CE5120701F1C8F0073F4C
:101010008CE5180739F507E225EE46EE67EF7CE52B
:1010200005C007E225EE45EE69ED7CE5C7010E94AB
:10103000AC1FECC406E221EE40EE64EF7CE5F6CF97
:1010400007E225EE44EE65EF7CE5F0CF06E221EE07
:1010500042EE66EF7CE5EACF08E221E045EE6AED7C
:101060007CE5E4CFF7018281882309F45BC110920B
:101070006B040430FDE51F0758F40B3F2CE5120705
:1010800080F4C80182509C45449708F035C109C0DE
:1010900002363DE5130729F0063A8DE5180709F0F9
:1010A0002BC10E94411790937804809377040131FB
:1010B0009CE5190709F4C6C008F042C00930FCE5F8
:1010C0001F0709F49BC000F505303CE5130709F440
:1010D00085C078F403309CE5190709F478C008F05E
:1010E0007AC002301C4509F0F7C080917704816016
:1010F000F1C007302CE5120709F478C008F07AC077
:10110000809177048061E6C00D308CE5180709F402
:1011100087C058F40B30ECE51E0709F479C008F0DD
:101120007BC08091770488606FC00F302CE5120778
:1011300009F480C008F082C080917704877FCAC01C
:101140000E3F8CE5180709F471C000F50531ECE598
:101150001E0709F485C068F403312CE5120709F471
:1011600075C008F095C00E94592A809177048F7746
:10117000B1C00C3F8CE51807A9F108F054C00B3F33
:101180001C4509F0A9C08091780440C00230FDE5FB
:101190001F0709F489C058F401153DE5130709F448
:1011A0005AC008F069C08091780482602FC002366E
:1011B0009DE5190709F47EC0063AEDE51E0709F41E
:1011C00083C003301D4509F087C060E06EC0809188
:1011D000770482607FC08091770416C08091770485
:1011E000886078C08091780482604FC080917704D5
:1011F000806270C08091770480646CC00E94592A1C
:1012000080917704806866C0846064C081603DC05E
:10121000809177048E7F5EC0809177048D7F5AC065
:101220008091770416C08091780418C0809178046A
:101230008D7F2BC0809177048F7E4CC08091770486
:101240008F7D48C0809177048F7B44C08091770464
:10125000877F8B7F3FC0809178048D7F8E7F15C004
:101260008091770482FB222720F991E0922790FB5E
:1012700082F990FB83F92EC080917804982F909585
:1012800091708E7F892B90FB81F98093780424C024
:101290000E94592A8091770487FB222720F991E048
:1012A000922790FB87F916C061E08EE090E00E94E3
:1012B000C33112C08091770484FB222720F991E08A
:1012C000922790FB84F906C080917704982F90951F
:1012D00090FB80F9809377046091770410917804F3
:1012E00084E090E00E94C331612F82E290E00E948E
:1012F000C3310E94592A8AC306312CE5120721F511
:1013000080914E078A7A91E009F490E090930C0264
:10131000882311F065E301C069E286EB96E00E9444
:101320003B1F0FC00631FCE51F0709F040C080914C
:101330000C02882309F48DC365E386EB96E00E94D6
:10134000131F0E94502662C30B353DE5130749F178
:1013500058F401159CE51907B1F00F3D1C4509F043
:1013600042C00E94521752C30C35FDE51F07D9F049
:101370000D351D45C1F58091780482FB882780F9E1
:1013800091E0892711C00E94592A3FEF84E39CE035
:10139000315080409040E1F700C000000E948C1E58
:1013A00035C381E001C080E00E94112A1CC08091F9
:1013B0004E0782720D3C2CE5120709F4D7C308F0E2
:1013C0007AC3073C9CE5190709F4BCC308F051C374
:1013D000043CFCE51F0709F4ABC308F03CC3033C25
:1013E0001C4509F4F0C2F70182810081D180882375
:1013F00059F0802F9D2D0E943627182F682F802F9F
:101400009D2D0E94992905C0802F9D2D0E946C2939
:10141000182F20E3129FF001112436E0D39EE00D37
:10142000F11D1124E00FF11DEE0FFF1FE75CF64FD9
:10143000859194910E94A7158C01982EF701D28076
:10144000A580A2943FE0A32280912C078770B9F079
:10145000DD20A9F0812F807F803421F080E2800F91
:10146000883068F08091780482FD09C082E00E9493
:10147000F42980912C078770CC24C3948111C12C4E
:10148000B12EB2949FE0B9228B2D90E08C30910563
:1014900008F05CC2FC01EA5AFF4F0C948832812F9D
:1014A000807F1F70882311F01295107FDD20B9F026
:1014B000112309F438C280E2800F883010F09110B7
:1014C00006C080914E07182B10934E0705C08091DF
:1014D0004D07182B10934D070E94502624C2802FD1
:1014E0000E940F06112309F431C2005E083078F122
:1014F000992069F1109580914D07182310934D079D
:1015000029C0812F807F1F70803211F01295107FCB
:10151000992021F0F1E09F16D9F149C0809178041B
:1015200082FF1BC0DD2069F0112339F080914E0746
:10153000182B10934E070E94502680E00E9441060F
:1015400005C280E00E940F06112309F4FFC1812F1C
:101550000E9449260E945026F9C1DD2081F0809129
:101560004F07AA2051F001E0A01207C0182B18174E
:1015700009F4ECC110934F07E9C1812B10C0AA20D8
:1015800021F021E0A21609F4E1C10E94432627C000
:10159000DD2041F035E03A1508F4D8C1812F0E94D2
:1015A0000506D4C184E08A1508F4D0C118C0DD2036
:1015B00049F0AA2099F3F701858180FFB4C18F70AB
:1015C0008583ECCFAA2059F0093309F0BCC1FFEFA5
:1015D00017EE23E0F15010402040E1F7B2C1812F17
:1015E0000E94FE05B3C1812F86958695837019F000
:1015F000813059F0ABC1DD2019F0C801937002C0F1
:1016000080E090E00E94861FA7C1DD2019F0C8018C
:10161000937002C080E090E00E94701F9DC1802FF7
:10162000DD2019F00E948B2D02C00E94D22C0E9456
:10163000E62D92C1812F837009F069C0D1108AC153
:10164000902F929596959770990F990F802F8F7084
:10165000882E912CA12CB12C092E04C0880C991C29
:10166000AA1CBB1C0A94D2F704FF12C04FE050E042
:1016700060E070E004C0440F551F661F771F9A9505
:10168000D2F7DB01CA0180959095A095B09503C073
:1016900080E090E0DC0116951695412F43704230B2
:1016A00019F1C8F400917102109172022091730235
:1016B00030917402413059F088299929AA29BB290F
:1016C000BC01CD0160237123822393230AC0802AA9
:1016D000912AA22AB32ABC01CD01682979298A2935
:1016E0009B290E944F2A36C188299929AA29BB29FA
:1016F0000091710210917202209173023091740274
:10170000BC01CD016027712782279327EACFDD2016
:1017100019F0812F817001C08695882309F41AC1C0
:10172000902F929596959770990F990F802F8F70A3
:10173000882E912CA12CB12C092E04C0880C991C48
:10174000AA1CBB1C0A94D2F704FF12C04FE050E061
:1017500060E070E004C0440F551F661F771F9A9524
:10176000D2F7DB01CA0180959095A095B09503C092
:1017700080E090E0DC0116951695412F43704230D1
:10178000D9F068F5009130021091310220913202B7
:1017900030913302413059F088299929AA29BB296F
:1017A000BC01CD0160237123822393231EC0802AB4
:1017B000912AA22AB32A13C088299929AA29BB29C8
:1017C00000913002109131022091320230913302A7
:1017D000BC01CD01602771278227932706C0BC0179
:1017E000CD01682979298A299B290E94C529B2C07F
:1017F0001F70DD2039F0812F0E942E2A802F0E9439
:101800000506A8C0802F0E94FE05812F0E94CF29C7
:10181000A1C0802F32EF931609F443C0391538F078
:1018200090EF991659F0E1EF9E16B1F177C0F3EF02
:101830009F16F1F124EF921659F170C0DD2019F1D5
:1018400034E03A1508F482C01F7181E090E0A0E016
:10185000B0E0AC01BD0104C0440F551F661F771FE7
:101860001A95D2F78091300290913102A091320204
:10187000B09133028A019B01082719272A273B27A9
:10188000C901B80129C025E02A1508F45FC0DCCFE2
:101890008091780482FF23C0DD2029F0812F8F7191
:1018A00030C0DD20D9F3812F8F710E94CF294EC027
:1018B000DD2079F01F7181E090E0A0E0B0E0BC0194
:1018C000CD0104C0660F771F881F991F1A95D2F7A4
:1018D00003C060E070E0CB010E94C52937C0DD2065
:1018E00099F01F71812F0E942E2A8091780482FD29
:1018F00007C038E0139FC0011124836080932C0738
:10190000812F0E942E2A22C081E00E94F42981E0CA
:101910008A15E0F482E00E94F42918C0DD2029F045
:10192000AA2009F4BBCF802F09CEAA2009F4BBCF8F
:10193000893349F49FEFE7EEF3E09150E040F04047
:10194000E1F700C00000802F0E940F0688EF8B0D8A
:10195000843010F40E949C1FCC20A9F080912C07A9
:1019600080FD11C0F70112828595859585950E94AD
:101970002E2AC7010E94610780912C0785958595C5
:1019800085950E94CF2985E0F701DE01119601902F
:101990000D928A95E1F789819A810E946C299A813A
:1019A00000E3809FF001112416E0919FE00DF11DEE
:1019B00011248981E80FF11DEE0FFF1FE75CF64F40
:1019C00085919491F4C080915E0480FFABC08E7FBE
:1019D00080935E0460915E0470915F048091600466
:1019E000909161040E94EF2A0E94BF208091AA0278
:1019F00081608093AA020FEF10E722E001501040AF
:101A00002040E1F700C000000E946E2A80912C0760
:101A1000877009F4CCC0F7018281882309F4C7C01C
:101A20008091780482FDC3C082E02A960FB6F894B4
:101A3000DEBF0FBECDBFDF91CF911F910F91FF9001
:101A4000EF90DF90CF90BF90AF909F908F900C94CD
:101A5000F42969E272CC053C9CE5190709F46DC0D4
:101A6000063C1C4509F0BFCC46EA5CE26FEA7CE22A
:101A700081C00A3CFCE51F0709F46EC070F4083C05
:101A80003CE5130709F463C0093C1C4509F0ABCCE5
:101A90004AE95CE26EE87CE26DC00B3CECE51E07B7
:101AA00009F45FC00C3C1C4509F09DCC41E05BE2B1
:101AB00062E17BE25FC0023D2CE5120709F466C0DB
:101AC00098F40F3C8CE5180709F45AC008F455C087
:101AD000003DECE51E0709F456C0013D1C4509F028
:101AE00082CC6EE089E060C0053D2CE5120709F468
:101AF00053C060F4033D8CE5180709F44AC0043D67
:101B00001C4509F070CC61E088E14BC0063DECE576
:101B10001E0709F444C00E351D4509F064CC6AE285
:101B200085E242C0816080935E0461E0869539C0A1
:101B300040E55EE269E57EE21DC049E55EE260E502
:101B40007EE218C04FEA5CE266EA7CE213C04EE82F
:101B50005CE26AE97CE20EC046E75CE262E87CE2B5
:101B600009C042E85CE266E77CE204C042E15BE275
:101B700061E07BE20E94B92049CF61E081E011C0C1
:101B800065E082E011C068E086E00EC064E18FE0AD
:101B90000BC067E185E108C062E289E105C061E050
:101BA00083E20E94102E32CF0E94A7202FCF2A96C8
:101BB0000FB6F894DEBF0FBECDBFDF91CF911F915E
:101BC0000F91FF90EF90DF90CF90BF90AF909F90DC
:101BD0008F900895CF93DF93CDB7DEB762970FB69E
:101BE000F894DEBF0FBECDBF84B7877F84BF0FB62A
:101BF000F894A895809160008861809360001092AD
:101C000060000FBE90E080E80FB6F894809361000A
:101C1000909361000FBE85B7806885BF85B78068E7
:101C200085BF8FE593E190930B0280930A020E9497
:101C3000EC240E940B258091E20084608093E200F6
:101C400078948091A1048823A1F01091E9001F707D
:101C50009091EC00892F817090FD80E8182B1092F4
:101C6000E9008091E80083FD0E94DB211F70109342
:101C7000E90082E084BD93E095BD9AEF97BD809323
:101C80006E0010920D0210920E0210920F0210922E
:101C900010020E94FA1480930401809104018823A9
:101CA00021F0109246018BE103C08BE18093460145
:101CB000809347010E94FA1481110E94CF2F8091D6
:101CC000040180910401811102C094E001C090E000
:101CD00090931A0284E0891B8093190209E911E0AC
:101CE0008DE9E82E81E0F82ED8018D918D018F3F8E
:101CF00011F00E949015E016F106B1F70DE911E020
:101D0000B3EAEB2EB1E0FB2EF80181918F018F3FFA
:101D100011F00E949015E016F106B1F788E0ECE1B1
:101D2000F2E0DF01282F1D922A95E9F7E1E1F2E0C8
:101D3000DF011D928A95E9F780E090E00E94BD31B5
:101D4000893E9E4F11F00E94521782E090E00E945F
:101D5000AF31809324020E944117909378048093BE
:101D600077040E94C617EFE3FCE93197F1F700C052
:101D700000000E94C6170E94FA14811102C0E4E01C
:101D800001C0E0E0F0E0E45EFD4F808181FF08C02B
:101D90006FEF7FEF80E090E00E94E1310E948C1EA7
:101DA00083E090E00E94AF31682F70E080E090E027
:101DB0000E944F2A0E94FA14882311F080E001C08B
:101DC00082E080936C0280E88093AB040E94632ED3
:101DD0006DE070E089E091E00E946F21892B09F0AD
:101DE00043C080916C0263E070E081FD3AC086E000
:101DF00091E00E946F21892BB9F56DE070E086EFCC
:101E000090E00E946F21892B79F50E94D21EDC019F
:101E1000CB01805A9541AF4FBF4F8093630490939D
:101E20006404A0936504B0936604EEEAF4E080E0F5
:101E300092E0DF019C011D9221503040E1F7F093C8
:101E4000B506E093B4068FEF9FEF9093AD048093B7
:101E5000AC0481E0809368048093670410926D0263
:101E600003C083E091E0C5CF80911B0281113BC08C
:101E700080E090E00E94BD31893E9E4F21F00E949B
:101E800052170E94232B88E090E00E94B7316093A4
:101E90005E0470935F04809360049093610480916A
:101EA000AA0283608093AA026E7F71F40E94232BA2
:101EB00088E090E00E94B73160935E0470935F0405
:101EC00080936004909361040E94D52A0E94BF20F1
:101ED00080915E0480FF04C060E086950E94102E11
:101EE00081E080931B020E94FA14811102C00E94BB
:101EF000D22F85E091E090936F0480936E04F8E117
:101F00002F2E312C44244394512C8091A1048530F0
:101F100009F045C000E112E18091A104853009F08B
:101F20003AC08091A104843021F10E9437201092A0
:101F3000720440E40FB6F894A895209260000FBE9A
:101F40004093600083B7817F846083BF83B78160E3
:101F500083BF7894889583B78E7F83BF0FB6F8943C
:101F6000A895809160008861809360001092600065
:101F70000FBE8091A004882309F4CECF0E94C6171B
:101F8000ECE1F2E0819181117AC384E292E08E1754
:101F90009F07C1F7C1CF0E94592A0E949C1F0E942F
:101FA000C617D82E81110E94D21EACE1B2E0E5E244
:101FB000F2E000E010E0B02ECD9081918C2549F147
:101FC000E12CFF24F3949F2D9823F1F00E94FA1442
:101FD000882399F0EF82B886CF2081E009F480E071
:101FE00089870E94DE1E8160782F9B878A874F81B8
:101FF000588569858B850E94B906F801EB5DFD4F18
:102000008081F826F0821AC0E394FF0C96E0E91272
:10201000DACF0F5F1F4F0830110569F68FEF8C87FD
:102020008D871E860E94DE1E8160782F988B8F8799
:102030004C855D856E8588890E94B9060E94FA14D8
:102040008091A902882309F4CFC08091A802E09171
:102050005E04E695E81BE093A402823059F4F0E0B8
:10206000E95DFE4FE4910E2F10E0E3E9EE2EEDE185
:10207000FE2E6BC0863059F4F0E0EC5DFE4FE4912B
:102080000E2F10E073E8E72E7DE1F72E5EC0893059
:1020900061F4E695F0E0EF5DFE4FE4910E2F10E065
:1020A00061E3E62E6CE1F62E50C08F3061F4E695C8
:1020B000F0E0E25EFE4FE4910E2F10E055E9E52ED0
:1020C0005BE1F52E42C0853159F4F0E0E55EFE4F4C
:1020D000E4910E2F10E04FE0E42E4BE1F42E35C0DA
:1020E0008831F9F0833249F4E9E1F1E00591149186
:1020F00033E4E32E3DE1F32E28C08432C9F085326B
:10210000F1F48E2F63E00E945A32E92FF0E0EA5E8C
:10211000FE4FE4910E2F10E02CE6E22E2CE1F22E81
:1021200014C008E210E09CE7E92E9AE1F92E0DC0F8
:1021300004EF11E08DE3E82E8AE1F82E06C000EDF1
:1021400017E0B9EAEB2EB9E1FB2E8091A5028823B6
:1021500061F01092A5020E94BD179093A302809394
:10216000A2021092A7021092A6020E94BD17E0914F
:10217000A202F091A3029C012E1B3F0B2F3F3F4771
:1021800098F520912F022223B1F010922F02209176
:102190002D0230912E02821B930B8F3F9F4758F4E4
:1021A000205D3A4830932E0220932D028091AA029E
:1021B00088608093AA02A090A602B090A7020E0F9A
:1021C0001F1F1093A3020093A20282EA92E0F7017C
:1021D00009958091A6029091A702892B29F4AB283A
:1021E00019F081E080932F0280916804882309F41C
:1021F00056C180916E0290916F020E94C31EC297D9
:1022000008F44DC00E94DE1E90936F0280936E0210
:102210008EEA94E09093B5068093B4060E94FA1477
:102220008823C9F186E491E00E9461218091300207
:1022300090913102A0913202B09133028F3091051A
:10224000A8F4FC01EE59FF4F0C9488328EE391E024
:1022500008C088E391E005C082E391E002C08BE210
:1022600091E00E94612181E00E947720E4E3F2E0A6
:1022700001900020E9F78F0101501109A4E3EA2E33
:10228000A2E0FA2EE016F10650F4D7018D917D01FF
:102290000E94E120F7CF8EE491E00E9461218091BD
:1022A0006804882309F4E0C02091AC043091AD04A7
:1022B0002115310509F4D8C080916D028111D4C077
:1022C000082F10E07201082E02C0EE0CFF1C0A94C9
:1022D000E2F7A9014E215F21452B11F48F5FF0CF6A
:1022E00090916C029801F5E0220F331FFA95E1F707
:1022F00090FD12C08295880F807680931301220F83
:10230000232F221F330B319520931601815E80937A
:1023100014011092170112C075E0369527957A9531
:10232000E1F7220F220F220F2093130110921601C2
:10233000295F2093140183E08093170124E630E0A5
:1023400047E050E061E171E088E70E941A2F892B95
:1023500009F08AC080916C0280FD22C0A80165E06E
:10236000440F551F6A95E1F742555B4F04E610E0B4
:1023700020E230E060E488E70E94412F892B09F0D9
:1023800073C00E945120E094F0948091AC0490912D
:10239000AD04E822F922F092AD04E092AC0464C0EE
:1023A00080E2ECE4F2E0DF011D928A95E9F7A801F2
:1023B00035E0440F551F3A95E1F7E7EAF1E0FA8B73
:1023C000E98B03EA11E0A989BA898D91BA8BA98BAF
:1023D000F80191918F01BA01690F711D62557B4F10
:1023E00090E0845B9D4FFC0127E0922E9F01281B0B
:1023F000390B742C01C0770C2A95EAF75B01812C0C
:10240000D501CD905D01C720292D28192770622E96
:10241000022E000C330BBC2D01C0BB0F6A94EAF7EF
:102420006B2E3195219531092770332701C0C69451
:102430002A95EAF76C28C0806C286082839428E093
:102440008212DECF9A9431963FEF9312CFCF8989D3
:102450009A898B5A914009F0B6CF04E610E020E249
:1024600030E04CE452E086CF809167048823B9F0D5
:102470000E94D21E009163041091640420916504AF
:1024800030916604DC01CB01801B910BA20BB30BD6
:102490008F3F9F4FAF4FBF4710F40E943720D1109E
:1024A0000E94512086E0E7E5F7E0DE0111960190F9
:1024B0000D928A95E1F7E0905907F0905A07009144
:1024C0005B0710915C071092590710925A071092FF
:1024D0005B0710925C07E11003C0FF2009F451C0B4
:1024E00080915507909156070E94C31E9C019091C0
:1024F0005107992309F4D9C02531310508F441C0A9
:102500009F3F19F09F5F90935107EE2061F00E946A
:102510006B2D1E1414F09FEF01C091E0899F802D58
:10252000112480935907FF2061F00E946B2D1F1426
:1025300014F09FEF01C091E0899F802D11248093BA
:102540005A07309159073323E1F020915A0722238B
:10255000C1F045EB3403C0011124992319F0909385
:10256000590703C081E08093590735EB2303C0016D
:102570001124992319F090935A0703C081E08093A6
:102580005A07011103C0112309F451C08091530768
:10259000909154070E94C31E9C019091500799236B
:1025A00009F488C02135310508F441C09F3F19F076
:1025B0009F5F90935007002361F00E94492D1016F1
:1025C00014F09FEF01C091E0899F802D112480932A
:1025D0005B07112361F00E94492D111614F09FEF43
:1025E00001C091E0899F802D112480935C07309178
:1025F0005B073323E1F020915C072223C1F045EB18
:102600003403C0011124992319F090935B0703C090
:1026100081E080935B0735EB2303C00111249923EC
:1026200019F090935C0703C081E080935C07809170
:10263000590781110BC080915A07811107C0809101
:102640005B07811103C080915C0781110E94E62D18
:10265000EB82FC820D831E8386E0FE013196A7E5A6
:10266000B7E001900D928A95E1F70E949C1F90912E
:102670007002891709F449CC8093700246CC09BDD9
:1026800019BD09B400FEFDCF8091D8008F7D8093E5
:10269000D8008091E00082608093E0008091E000AB
:1026A00081FDFCCF0E94592A37CC2B30310508F030
:1026B00029CF67CF2B30310508F07ACFB8CF80E033
:1026C00008959091770492FF0DC0282F287128302B
:1026D00019F4877F846006C0282F2471243011F4F8
:1026E0008B7F886093FF0DC0282F2871283119F443
:1026F000877E846106C0282F2471243111F48B7EDB
:1027000088612091780420FF0DC0382F387138304F
:1027100019F4877F816006C0382F3171313011F490
:102720008E7F886021FF0DC0282F2871283119F471
:10273000877E816106C0282F2171213111F48E7EA0
:10274000886194FD877E0895AF92BF92CF92DF9209
:10275000EF92FF920F931F93CF93DF937C015B0166
:102760006A018091A1028A3018F001E010E002C0F5
:102770000AE010E0C1E0D0E0F894B501C701F6012D
:1027800009957894811115C021960C171D0794F0B6
:10279000CC9F9001CD9F300D300D112480E090E052
:1027A00045E34A95F1F70000019682179307C1F7B8
:1027B000E3CF81E0DF91CF911F910F91FF90EF90D8
:1027C000DF90CF90BF90AF900895CF93DF93CDB7B8
:1027D000DEB728970FB6F894DEBF0FBECDBF85E0F9
:1027E000EEE5F4E0DE01119601900D928A95E1F795
:1027F0008091A8029091A902A091AA028E839F8342
:10280000A887288540919D0250919E0260919F0269
:102810007091A0023FB7F894809173049091740472
:10282000A0917504B09176043FBF841B950BA60B55
:10283000B70B84369105A105B10510F4222319F1D7
:10284000809131019091320184579D4F4091300128
:1028500050E04930510510F048E050E0BE016F5F94
:102860007F4F0E94B73283E090E00E94BB30882304
:1028700069F00E94D21E60939D0270939E02809325
:102880009F029093A0021092AA0281E028960FB6B0
:10289000F894DEBF0FBECDBFDF91CF910895EF92C8
:1028A000FF921F93CF93DF9300D000D01F92CDB73C
:1028B000DEB77B0180E090E00E94BB30882309F402
:1028C00063C040911B0150E04115510511F041E0FA
:1028D00050E060911C0170911D0164577D4FCE0145
:1028E00005960E94B7324091840250918502609112
:1028F0008602709187022FB7F894809173049091AB
:102900007404A0917504B09176042FBF841B950BBD
:10291000A60BB70B84369105A105B10538F48DE8F7
:1029200092E00E9498219D81891781F181E090E0D9
:102930000E94BB30182F882391F04091230150E072
:102940004530510510F044E050E060912401709151
:10295000250164577D4FCE0101960E94B7328DE864
:1029600092E00E94982191E02D81281390E0192394
:1029700041F10E94D21E609384027093850280937D
:102980008602909387020FC010E001C011E0809191
:102990008D0290918E02A0918F02B0919002898356
:1029A0009A83AB83BC83112361F089819A81AB81C7
:1029B000BC818093800290938102A0938202B093A5
:1029C00083028091800290918102A0918202B09155
:1029D0008302F70180839183A283B383812F0F90B9
:1029E0000F900F900F900F90DF91CF911F91FF905C
:1029F000EF90089580917F02811118C08091D800D6
:102A000080618093D8008AE18A95F1F700C08091B7
:102A1000D90080FD02C082E001C081E080937F0286
:102A2000823021F40E94EC241092A10481E0909164
:102A30007F02913009F080E008950F931F930E9468
:102A4000FA14882321F01F910F910C94D21E0E943A
:102A5000D21E00910D0210910E0220910F023091B2
:102A60001002600F711F821F931F1F910F91089515
:102A7000CF93DF9300D000D0CDB7DEB7409188026E
:102A80005091890260918A0270918B022FB7F8945D
:102A90008091730490917404A0917504B0917604B0
:102AA0002FBF841B950BA60BB70B84369105A10590
:102AB000B10570F10E941D15DC01CB010296A11D2C
:102AC000B11D89839A83AB83BC8380912901909146
:102AD0002A0184579D4F4091280150E0453051050F
:102AE00010F044E050E0BE016F5F7F4F0E94B732AC
:102AF00082E090E00E94BB30882359F00E94D21EF1
:102B0000609388027093890280938A0290938B026B
:102B100081E00F900F900F900F90DF91CF9108956B
:102B2000F894E82FE295EF70F0E031A1282F2F7094
:102B300081E090E001C0880F2A95EAF7982F9095E0
:102B4000932391A392A1892B82A378940895CF9384
:102B5000DF938238910569F1B0F48133910509F46E
:102B60006FC048F48932910509F465C08A32910535
:102B700009F46BC08AC08533910509F457C08933C5
:102B80009105B9F082C0833E910571F138F4803E21
:102B90009105B1F0823E910511F177C0863E910515
:102BA000B9F1873E9105C9F1843E910509F06DC0E8
:102BB00024C02091770420FD53C021FD51C065C081
:102BC0008091770480FD46C08091780480FF48C0E2
:102BD0008091770484FD50C183EE90E04FC18091D5
:102BE000770482FF3AC0F4CF8091770482FD35C02C
:102BF0008091780480FD34C0EBCF8091780481FF10
:102C000035C08091770484FD37C187EE90E036C1EE
:102C10008091770483FF27C0F4CF8091770483FDF0
:102C200022C08091780481FD21C0EBCF8091770490
:102C300085FD1FC021C08091770485FD1DC019C08E
:102C40008091770486FD1BC01DC08091770486FDAE
:102C500019C015C089E390E011C182EE90E00EC169
:102C600080EE90E00BC186EE90E008C184EE90E02B
:102C700005C189E290E002C185E390E0FFC08AE2ED
:102C800090E0FCC081E390E0F9C0811531E5930745
:102C900008F069C0811540E59407F0F09C0174E0EC
:102CA000369527957A95E1F7922F9370482F4370C8
:102CB00021E030E002C0220F331F4A95E2F73C6862
:102CC000392B982F9F709695969540E2949FC0015E
:102CD0001124822B932BD2C0883E910568F5803E4B
:102CE000910508F0CBC0883A9105B8F4853A910572
:102CF00048F0855AE82FF0E0E555FE4F808190E0DE
:102D00009064BCC08130910509F4B3C008F4B4C02C
:102D10008430910508F4B0C0B1C08F3B910508F034
:102D2000ABC0885AE82FF0E0EE0FFF1FE255FE4FD0
:102D3000808191819464A2C0811520E2920758F4A9
:102D4000811531E0930708F099C08D3E910508F494
:102D500093C0906593C0811540E4940708F48CC03B
:102D60009F70906A8BC0811525E5920708F042C0DC
:102D7000811534E5930728F0982F8827846F906A8F
:102D80007DC0811543E59407B0F09C012370332783
:102D900041E050E002C0440F551F2A95E2F7282F6A
:102DA0002695269580E2289F90011124CA01822B46
:102DB000932B9A6863C0811522E5920728F4982F17
:102DC0008827816F906A5AC09C012370332741E0A5
:102DD00050E002C0440F551F2A95E2F7282F269590
:102DE000269580E2289F90011124CA01822B932B03
:102DF0009C6844C0EC01811539E59307A8F481155E
:102E0000984528F09C2F8827806F906A37C0C1159D
:102E100086E5D80788F58C2F0E9461138F7190E0AA
:102E2000982F882790622AC081152AE5920790F48E
:102E30008C2F8F700E94611394E0D695C7959A9558
:102E4000E1F7CF70D0E0DC2FCC27D0699E01282B92
:102E5000C90114C090568115904270F48D2F8F7166
:102E60000E946113282F2F71CE0199279062922B17
:102E700005C081E090E002C080E090E0DF91CF915A
:102E80000895CF9384E090E00E94AF31C82F82E292
:102E900090E00E94AF312C2F30E0A901582BCA01DD
:102EA000CF91089569EE7EEF80E090E00E94E131DD
:102EB00060E082E090E00E94C33160E083E090E057
:102EC0000E94C3311092710210927202109273022A
:102ED0001092740260E084E090E00E94C33160E0F0
:102EE00082E290E00E94C33160E085E090E00E94C1
:102EF000C33160E086E090E00E94C3316FEF87E06D
:102F000090E00E94C33140E050E0BA0188E090E0D8
:102F10000E94D53160E08DE090E00E94C33140E036
:102F200050E0BA0188E190E00E94D53160E087E18D
:102F300090E00E94C33140E050E0BA018CE190E0A3
:102F40000E94D53160E070E080E290E00E94E131C3
:102F500040E050E0BA0188E190E00E94D53140E0C5
:102F600050E0BA018FE090E00E94D53140E050E09F
:102F7000BA0183E190E00C94D5310E94FA148111DA
:102F80000C94DE1E0E941D15CB0108957F928F9236
:102F90009F92AF92BF92CF92DF92EF92FF920F93E8
:102FA0001F93CF93DF93CDB7DEB72C970FB6F8946E
:102FB000DEBF0FBECDBFAE014F5F5F4F7A0188E02D
:102FC000DA011D928A95E9F709E911E06A018DE9B4
:102FD000A82E81E0B82E88248394912CF80180815A
:102FE0008F3F09F441C0F894E82FE295EF70F0E0CC
:102FF00021A18F70A40102C0440F551F8A95E2F7EA
:10300000CA01922F982B91A392A18095892382A324
:10301000789400C0EDE9F1E0712C31E021912F3F6F
:1030200089F0A22FA295AF70B0E090968C9190E0BD
:103030002F7002C0959587952A95E2F780FD02C012
:10304000832F01C080E0782A330F51E0E33AF5077F
:1030500029F7D8018C918F3F11F00E949015B0EAAA
:10306000BA95F1F7F60170820F5F1F4FFFEFCF1A8D
:10307000DF0AA016B10609F0B1CF48E050E0B70171
:1030800081E192E00E94AA328C01892B41F088E014
:10309000F701A1E1B2E001900D928A95E1F7F0907D
:1030A0001A020115110549F081E0809377020E9410
:1030B000DE1E9093760280937502809177028823BA
:1030C000B9F080917502909176020E94C31E059717
:1030D00078F0A1E1B2E0EF2DF0E0E45EFD4F85E194
:1030E00092E02D9121938A179B07D9F710927702CE
:1030F0000115110509F012C10E94FA14E0911A029B
:10310000882309F477C019861A861B861C860E2F21
:1031100010E0045E1D4F8091A1028A3058F44FE404
:1031200054E1BE01675F7F4FC8010E94A41388234A
:10313000A1F10AC080917802909179020E94C31E89
:10314000843F914060F73AC048E355E1BE01675FB4
:103150007F4FC8010E94A4138823F9F045EE53E184
:10316000BE01675F7F4FC8010E94A4138823A9F0A6
:103170001092A1028091190290E044E050E0BE015B
:10318000675F7F4F845E9D4F0E94AA3221E02093AB
:103190007E02892B01F500E0C3C08091A1028F3F20
:1031A00019F08F5F8093A1028091A1028A3010F301
:1031B0000E94DE1E909379028093780280917E02B5
:1031C000882349F3FE01399684E0DF011D928A9538
:1031D000E9F710927E02E0911902F0E0E45EFD4F03
:1031E00089859A85AB85BC8580839183A283B383CF
:1031F00001E096C0F0E0E45EFD4FF89484E0ADE8B5
:10320000B2E001900D928A95E1F78DE892E00E947C
:10321000982180938C027894F894C0909102D09079
:103220009202E0909302F090940280917A02909141
:103230007B02A0917C02B0917D02C816D906EA06F5
:10324000FB06D1F0C0927A02D0927B02E0927C021F
:10325000F0927D020E94FA1481110EC00E94D21ECB
:10326000C61AD70AE80AF90AC0920D02D0920E02D5
:10327000E0920F02F09210027894F89480919C02F0
:10328000882309F449C080FF24C090919502809161
:103290005E0490FF09C0816080935E0460E0892F26
:1032A00086950E94102E15C08E7F80935E040E942A
:1032B000BF208091AA0281608093AA02BFEFE0E75D
:1032C000F2E0B150E040F040E1F700C000000E94A1
:1032D0006E2A80919C0281FF09C020E040919802F3
:1032E00060919702809196020E94D42B80919C025B
:1032F00082FF09C080919B02882319F00E94C6209A
:1033000002C00E94BF2080919C0283FF03C081E025
:103310008093A50210929C02789402C001E010E014
:10332000802F2C960FB6F894DEBF0FBECDBFDF9175
:10333000CF911F910F91FF90EF90DF90CF90BF90B2
:10334000AF909F908F907F900895089580917E0414
:10335000089508958093790470937B0460937A04B0
:103360008091A104843001F582E08093E9008FEF21
:103370009091E800815095FD06C095ED9A95F1F782
:1033800000008111F5CF8091E80085FF0DC040E07D
:1033900050E063E070E089E794E00E94AF21809103
:1033A000E8008E778093E8000895BC0184E00C94D7
:1033B000AA19BC0183E00C94AA1922E02093E90029
:1033C0002FEF3091E800215035FD06C035ED3A95DC
:1033D000F1F700002111F5CF2091E80025FF0BC087
:1033E00040E050E066E070E00E94AF218091E8008C
:1033F0008E778093E8000895CF93DF9320914B015F
:10340000222339F02091770427FF03C060E222E0F5
:1034100002C068E021E02093E9002FEF3091E8003E
:10342000215035FD06C035ED3A95F1F70000211128
:10343000F5CF2091E80025FF1DC0EC0180914B01E4
:10344000811105C040E050E068E070E003C070E02A
:1034500040E050E0CE010E94AF218091E8008E77DD
:103460008093E80080E2FE01AFE7B4E001900D92A6
:103470008A95E1F7DF91CF9108950F931F93CF9332
:10348000DF93EC0100E010E080914A01282F30E04A
:103490000217130724F5909148019801290F311D57
:1034A000A901440F551F240F351F22553D4F869506
:1034B00090E04C81081719071CF4442331F002C036
:1034C000411103C04091610401C040E0609160047B
:1034D00080915F040E943B2B0F5F1F4FD5CF0E944E
:1034E0006E2A8C8190E00196817099278C83DF9100
:1034F000CF911F910F9108958F929F92AF92BF929B
:10350000CF92DF92EF92FF920F931F93CF93DF93AF
:103510008C01FC014481C42FD0E09E01DE010E9499
:103520004B329B01AC010E9416326B017C01E0E240
:10353000F0E0EC1BFD0BA5E5B0E09B01AC010E94A7
:1035400016324B015C019F01DF010E948E329B010C
:10355000AC010E9421329B01AC012C0D3D1D4E1D82
:103560005F1DC501B4010E942932C22FD22F2A3219
:1035700028F4F3E02F9F900111240DC025E530E0E1
:103580002C1B3109C901880F991F280F391F37FFDC
:1035900002C02F5F3F4F35952795C22FC095F12C64
:1035A00085E5E82EED1A80914A01F816C8F4F1FC81
:1035B00002C08E2D01C08D2F909148012F2D30E03B
:1035C000290F311DA901440F551F240F351F225506
:1035D0003D4F4C2F609160040E943B2BF394E3CF4E
:1035E0000E946E2AF8018481811102C091E003C01B
:1035F000803219F49FEF9093450190914501890F16
:10360000F8018483DF91CF911F910F91FF90EF908C
:10361000DF90CF90BF90AF909F908F9008951F93B1
:10362000CF93DF93EC018C81811109C081E08C8301
:103630001092AC0292E090934401809343018091F8
:10364000480190914901891770F4E82FF0E09F013B
:10365000220F331FE20FF31FE255FD4F118210823C
:1036600012828F5FF0CF10E060914A011617C0F50B
:10367000E12FF0E070E0CF010E9474322091480108
:10368000820F2091AC02022E000C330B90E0E21767
:10369000F307CCF020914401022E000C330B2E17BF
:1036A0003F078CF09C01220F331F820F931F9C0158
:1036B00022553D4F409161046091600480915F0408
:1036C0000E943B2B0BC0FC01EE0FFF1F8E0F9F1FB4
:1036D000FC01E255FD4F1182108212821F5FC4CFA0
:1036E0000E946E2A809143012091AC02280F209302
:1036F000AC0290914401980F9093440119165CF428
:10370000022E000C330B40914A0150E04150510908
:103710002417350734F0819580934301813009F4F3
:103720001C82DF91CF911F9108957F928F929F927B
:10373000AF92BF92CF92DF92EF92FF920F931F93BF
:10374000CF93DF93EC018A8180FF03C0BB24BA943E
:1037500002C0BB24B3948C8181110DC081E0B812EA
:1037600006C080914A0181508093AB0202C0109242
:10377000AB0281E08C83A12C46E3842E90904A0119
:10378000A91408F041C080914801CA2CD12C8601AF
:10379000080F111DC801880F991F080F191F025526
:1037A0001D4FF80111821082128234E0E32EF12CB9
:1037B000712C8091AB02870D87332CF0682D0E940D
:1037C0006632892F02C087FD890D082E000C990BE7
:1037D000C816D90691F4809161048E9DA0018F9D39
:1037E000500D112455954795559547959801609131
:1037F000600480915F040E943B2B7B0CF1E0EF1A88
:10380000F108B9F6A394BACF0E946E2A8091AB0258
:1038100091E0B9120EC0811107C080914A01815018
:103820008093AB021C820FC081508093AB02BC829C
:103830000AC090E0019660914A0170E00E947432E3
:103840008093AB028C83DF91CF911F910F91FF90FA
:10385000EF90DF90CF90BF90AF909F908F907F9030
:103860000895FF920F931F93CF93DF93EC01F12CF8
:103870000FEF10E060914A01F616F0F480914801D4
:103880002F2D30E0280F311DC901880F991F280FF7
:10389000391F22553D4F70E0C8010E947432962FA7
:1038A0008C814091610460916004F99E800D112427
:1038B0000E943B2BF394DECF0E946E2A9A818C816A
:1038C00090FF02C08F5F01C081508C83DF91CF9148
:1038D0001F910F91FF9008957F928F929F92AF92C8
:1038E000BF92CF92DF92EF92FF920F931F93CF93ED
:1038F000DF93FC018280748081E08483EEE8F1E054
:103900009490EDE0F2E0E491A12CF5E0BF2ECC2400
:10391000CA94D12CE9190E2F10E080914A01A81603
:1039200008F0A2C0EA2CF12C22E0281568F0BE9C19
:10393000F001BF9CF00D1124E05BFC4F80915F040F
:10394000808380916004818371100AC0BE9CF00165
:10395000BF9CF00D1124E05BFC4F138212826AC001
:10396000BE9CE001BF9CD00D1124C05BDC4F8B815D
:103970008823F9F081508B832FEF829FC00111249F
:103980006C8170E00E943631FB01FF27E257FE4F49
:103990008491E82FE9192FEFE29FC0011124B801AB
:1039A0000E94363180916104689FB00111247A83AE
:1039B00041C00E949631209161042695215830E043
:1039C000A901440F551F322F2227240F351F232F03
:1039D00033278217930774F582E0881588F40E94D4
:1039E0009631B6010E94743288830E9496312091EC
:1039F00060042695622F70E00E947432280F29839C
:103A0000BE9CF001BF9CF00D1124E05BFC4F1282C4
:103A100080916104843120F0893C18F088EC01C069
:103A200084E1BE9CF001BF9CF00D1124E05BFC4FD3
:103A300084838383809148019701280F311DC90138
:103A4000880F991F280F391F22553D4FBE9CF0014A
:103A5000BF9CF00D1124E05BFC4F428161818081AD
:103A60000E943B2BA39459CFDF91CF911F910F91CF
:103A7000FF90EF90DF90CF90BF90AF909F908F908E
:103A80007F900C946E2A0F931F93CF93DF9300D0F7
:103A90001F92CDB7DEB78C018091AD0281110AC0B3
:103AA0009E012F5F3F4F48E76FEF0E943B2B8A81BB
:103AB0008093AD02F8018481813051F028F082308A
:103AC00061F44091AD020AC08091AD0240E007C0B0
:103AD0006091AD0240E080E003C040E080E060E043
:103AE0000E94BA2AF801848190E0019663E070E0B8
:103AF0000E94743284830F900F900F90DF91CF91CA
:103B00001F910F910895CF93DF93EC01EEE5F4E060
:103B1000438162818C810E94B82C8C818F5F8C8361
:103B2000DF91CF910895CF93DF93EC01EC81F0E02A
:103B3000E257FE4F4491EEE5F4E0628181810E94FC
:103B4000B82C8C818F5F8C83DF91CF910895209169
:103B5000E4003091E50095E64091EC00842F8170FF
:103B600040FF23C08091E80080FD1DC08091A1042A
:103B7000882399F0853099F08091EB0085FD11C084
:103B80004091E4005091E5002417350729F3915046
:103B900011F09A01E1CF84E0089582E0089583E076
:103BA000089581E0089580E008954091E80042FF83
:103BB000DDCF08958091A30487FF11C08091E800B4
:103BC00082FD05C08091A1048111F8CF11C08091C0
:103BD000E8008B770BC08091A104882349F0809185
:103BE000E80080FFF8CF8091E8008E778093E800AE
:103BF0000895982F973068F59093E900981739F059
:103C00007091EC002091ED005091F00003C0242F42
:103C1000762F50E021FD02C09F5FECCF3091EB008A
:103C20003E7F3093EB003091ED003D7F3093ED000F
:103C30003091EB0031603093EB007093EC002093F7
:103C4000ED005093F0002091EE0027FDE5CF80E0DD
:103C500008958F708093E90081E008952091A90470
:103C60003091AA042617370748F06115710539F419
:103C70002091E8002E772093E80001C0B901FC01F3
:103C800020E06115710579F18091A1048823F1F19B
:103C90008530F1F18091E80083FD3CC08091E8001F
:103CA00082FD2EC08091E80080FFEBCF2091F300D1
:103CB0008091F20090E0922B6115710551F08830EF
:103CC000910538F421912093F1006150710901961A
:103CD000F3CF21E0089709F020E08091E8008E778B
:103CE0008093E800CECF2111CFCF0AC08091A104EC
:103CF000882361F0853061F08091E80083FD0AC07F
:103D00008091E80082FFF2CF80E0089582E008957C
:103D100083E0089581E0089587E797E7909301088D
:103D2000809300089AE088E10FB6F894A8958093F4
:103D300060000FBE90936000FFCF78941F920F92A7
:103D40000FB60F9211248F939F93AF93BF938091DF
:103D5000730490917404A0917504B0917604019657
:103D6000A11DB11D8093730490937404A0937504F6
:103D7000B0937604BF91AF919F918F910F900FBE3A
:103D80000F901F9018959C014FB7F8948091730481
:103D900090917404A0917504B09176044FBF821B7A
:103DA000930B08952FB7F894609173047091740485
:103DB00080917504909176042FBF08952FB7F894E1
:103DC0008091730490917404A0917504B09176046D
:103DD0002FBF08951F920F920FB60F9211248F9349
:103DE0009F93AF93BF9380917204811113C0809110
:103DF000730490917404A0917504B0917604419677
:103E0000A11DB11D8093730490937404A093750455
:103E1000B0937604BF91AF919F918F910F900FBE99
:103E20000F901F90189520914B012223C9F02091EB
:103E3000770427FF15C0262F2695269526952E3127
:103E4000C8F4FC01E20FF11D677081E090E001C051
:103E5000880F6A95EAF78095928189238283089575
:103E6000FC0106962281621301C012823196E81786
:103E7000F907C1F7089520914B012223C1F0209149
:103E8000770427FF14C0262F2695269526952E31D8
:103E900030F5FC01E20FF11D677081E090E001C098
:103EA000880F6A95EAF79281892B82830895FC0135
:103EB00032962FEF30E04191641789F02F3F19F4CB
:103EC000411101C0232F3F5F3630A9F72F3F39F052
:103ED000FC01E20FF11D27FDFA9562830895089514
:103EE00020917004309171042817390771F0909374
:103EF000710480937004E0916E04F0916F04309728
:103F000021F00084F185E02D0994089520916C043E
:103F100030916D042817390771F090936D048093E8
:103F20006C04E0916E04F0916F04309721F00680EC
:103F3000F781E02D099408950E94FA14882351F026
:103F4000E0916E04F0916F04309721F00190F081C0
:103F5000E02D099480E00895EF92FF920F93CF93A4
:103F6000DF93C42FD22FFC0182818823D1F04093AC
:103F70006B040E94DE1E90936A048093690480E2C1
:103F80008C0F883008F06DC0C77081E001C0880FC9
:103F9000CA95EAF7DF91CF910F91FF90EF900C94C3
:103FA000050680916B0448134BC080916904909181
:103FB0006A040E94C31E883C910508F041C0CD17D9
:103FC000C9F080E28C0F883040F4C77081E001C0F6
:103FD000880FCA95EAF70E94FE0580E28D0F8830AF
:103FE00048F481E09D2F977001C0880F9A95EAF7F9
:103FF0000E940506093319F0E12CF12C03C080E57D
:10400000E82EF12C802F0E944106E114F10451F0BA
:104010008FE99FE00197F1F700C0000091E0E91AF5
:10402000F108F3CF802F0E940F0680E28D0F8830B9
:10403000C0F4D77081E001C0880FDA95EAF70AC0B2
:1040400080E28C0F883068F4C77081E001C0880F6F
:10405000CA95EAF7DF91CF910F91FF90EF900C9402
:10406000FE05DF91CF910F91FF90EF900895809121
:10407000680490916704882389F0992369F062E0CD
:1040800070E080E992E00E946F21892B19F0809105
:1040900067040895109267049091670481E089276E
:1040A0000895809168048823F9F00E94D21EDC01F3
:1040B000CB01805A9541AF4FBF4F809363049093DB
:1040C0006404A0936504B093660480916704811131
:1040D0000BC062E070E08EE892E00E946F21892BB5
:1040E00019F481E080936704809167040895CF9369
:1040F000E82F2091B4063091B5062E5A34404091F5
:10410000AB04642F70E0C9010E943631481B842F34
:10411000EE2351F066E00E945A32C82FC150A8F039
:1041200080E20E94E120FACFA901480F511D4115FC
:10413000524018F080E020E030E0280F311D225579
:104140003B4F3093B5062093B406CF9108959091DC
:104150005E0490FF04C09695981740F003C081114B
:1041600005C090E0961710F40C94592E61E00C9461
:10417000102E882311F0FA0101C0FB010994E8EA2E
:10418000F2E01182828184608283089560915E04EE
:10419000669570E04BE050E088E391E00E949D322C
:1041A000892B19F481E08093A9020E94BD17909396
:1041B000A3028093A2028091AA0284608093AA0243
:1041C0000895CF93DF938A3011F481E003C08D30DE
:1041D00029F480E0DF91CF910C947720682F8091B3
:1041E000B4069091B50626E0FC01AEEAB6E0019077
:1041F0000D922A95E1F7603E30F026E0FC01119225
:104200002A95E9F70AC0F6E06F9FB00111246750C4
:104210007C4F46E050E00E94A631C091B406D09198
:10422000B50646E050E0BE018EEA96E00E94AA3252
:10423000892B49F19E012E5A3440A90185E05695FB
:1042400047958A95E1F781E090E0BC0102C0660FD6
:10425000771F4A95E2F74091AC045091AD04462B8C
:10426000572B2B5F3F4F65E0369527956A95E1F711
:1042700002C0880F991F2A95E2F7842B952B909303
:10428000AD048093AC049E01285A34404091AB04A5
:10429000642F70E0C9010E943631481B463010F48B
:1042A000240F311D211582E0380710F020E030E0A6
:1042B00022553B4F3093B5062093B406DF91CF9142
:1042C0000895CF93DF93EC01FE018491882321F0C0
:1042D0000E94E1202196F8CFDF91CF910895EF92CF
:1042E000FF920F931F93CF93DF93EC017B0164E662
:1042F00070E088E70E94692E8C01EC0EFD1ECE1541
:10430000DF0561F017FD0AC0FE01849164E670E0EC
:104310000E94EA2E8C012196892B89F30E946E2F30
:10432000C801DF91CF911F910F91FF90EF900895F9
:10433000FC01AC014C5F5F4F8FEF91E3219182272D
:1043400028E030E087FF03C0880F892701C0880F6D
:1043500021503109B9F7E417F50781F70895EF9275
:10436000FF920F931F93CF93DF937C018B010E94E9
:10437000A71D811119C0E70101151105A1F0809158
:10438000E80085FD0AC08091E8008E778093E80000
:104390000E94A71D882381F307C089918093F100B3
:1043A00001501109E9CF80E0DF91CF911F910F916A
:1043B000FF90EF9008951F93CF93DF93CDB7DEB7B3
:1043C000AA970FB6F894DEBF0FBECDBFE3EAF4E0C4
:1043D0008BEA94E02091F10021938E179F07D1F78B
:1043E0008091A404833009F461C030F4813071F00D
:1043F000823009F49BC0B2C08A3009F487C08B3088
:1044000009F46CC0893009F0A9C020C08091A304D0
:10441000813A09F0A3C08091E800877F8093E8008B
:104420008091A7049091A804892B21F460E28FE782
:1044300094E003C060E080E090E070E00E942E1EF7
:104440008091E8008B778093E80088C08091A30476
:10445000813209F083C08091A7049091A80402974B
:1044600008F07CC08091E800877F8093E80080910D
:10447000E80082FD05C08091A1048111F8CF6EC0D3
:104480002091F3008091F20090E0922B029731F49A
:104490008091F100813011F0863021F48091F1009B
:1044A00080937E048091E8008B7754C08091A304B0
:1044B000813A09F053C08091A7049091A804892BF8
:1044C00009F04CC08091E800877F8093E8008091DC
:1044D000E80080FFFCCF80914B0137C08091A3049E
:1044E0008132E1F58091A7049091A804892BB1F560
:1044F0008091E800877F8093E8000E94DA1D809118
:10450000A50480934B010E94592A28C08091A304DE
:10451000813221F58091E800877F8093E8000E9436
:10452000DA1D8091A60480937D0418C08091A304B5
:10453000813AA1F48091E800877F8093E800809120
:10454000E80080FFFCCF80917D048093F100809192
:10455000E8008E778093E8000E94DA1D8091E800E1
:1045600083FFCEC18091A3049091A404492F50E011
:104570004A30510508F0C4C1FA01EF58FF4F0C94BE
:104580008832803821F0823809F0BAC108C08091A1
:104590009F049091A004992389F082600FC08091BC
:1045A000A7048F70873008F0ABC18093E900809139
:1045B000EB0085FB882780F91092E9009091E800D4
:1045C000977F9093E8008093F1001092F10065C10D
:1045D000282F2D7F09F094C1882319F0823061F0D3
:1045E0008FC18091A504813009F08AC1933009F010
:1045F00080E08093A0042EC08091A50481112AC080
:104600008091A7048F702FEF280F263008F078C113
:104610008093E9002091EB0020FF1CC0933021F42F
:104620008091EB00806214C09091EB0090619093B8
:10463000EB0021E030E0A90102C0440F551F8A952C
:10464000E2F74093EA001092EA008091EB00886064
:104650008093EB001092E9008091E800877F20C1F1
:1046600081114EC11091A5041F778091E3008078DD
:10467000812B8093E3008091E800877F8093E8009E
:104680000E94DA1D8091E80080FFFCCF8091E3005A
:1046900080688093E300111102C082E001C083E0D2
:1046A0008093A1042DC18058823008F029C18091E7
:1046B000A5049091A6048C3D53E0950779F583E01D
:1046C0008A838AE289834FB7F894DE01139620E04B
:1046D0003EE051E2E32FF0E050935700E49120FFD9
:1046E00003C0E295EF703F5FEF708E2F90E0EA30ED
:1046F00010F0C79601C0C0968D939D932F5F243113
:1047000049F74FBF8091E800877F8093E8006AE215
:1047100070E0CE0101960E942E1EAEC04091A7040B
:104720005091A804292F332723303105A9F068F4CC
:104730002130310509F4F3C02230310509F0E0C021
:104740008BE390E0E8E8F3E044C02132310521F149
:104750002232310571F1D4C0992781309105A1F041
:1047600058F0029709F0CCC0E5EDF3E0E4918E2F0C
:1047700090E0E5EDF3E02AC0E5EFF3E0E4918E2F61
:1047800090E0E5EFF3E022C0E3EEF3E0E4918E2F5A
:1047900090E0E3EEF3E01AC04115510509F4C4C0FE
:1047A0004130510509F0ACC089E090E0E3EBF3E063
:1047B00010C04115510509F4BCC04130510509F044
:1047C0009FC086EB90E0E2E9F2E003C0009709F4B5
:1047D00097C02091E800277F2093E8002091A9044A
:1047E0003091AA048217930708F49C0140E0211538
:1047F000310589F18091A104882309F43DC08530F9
:10480000D9F18091E80083FD37C08091E80082FDF6
:104810002FC08091E80080FFEACF4091F3008091A3
:10482000F20090E0942B2115310559F08830910564
:1048300040F444914093F1003196215031090196A2
:10484000F2CF41E0089709F040E08091E8008E77D0
:104850008093E800CCCF4111CDCF0AC08091A10454
:10486000882351F0853041F08091E80083FD04C039
:104870008091E80082FFF2CF8091E8008B778093EF
:10488000E8003EC08038E1F58091E800877F8093A2
:10489000E8008091A2048093F1008091E8008E7777
:1048A0008093E8000E94DA1D2BC0811129C08091FD
:1048B000A5049091A6049927029714F58091E80029
:1048C000877F8093E8001091A5041093A2040E94B2
:1048D000DA1D111106C08091E30087FD02C081E05E
:1048E00001C084E08093A10442E061EC81E00E9479
:1048F000F91D42E261EC82E00E94F91D8091A10461
:104900008091E80083FF1AC08091E800877F809340
:10491000E8008091EB0080628093EB000FC082E1A1
:1049200090E0E3ECF3E055CF89E090E0EAE9F3E0D2
:1049300050CF80E490E0E8E4F3E04BCFAA960FB6C6
:10494000F894DEBF0FBECDBFDF91CF911F910895C8
:104950001F920F920FB60F9211242F933F934F93F4
:104960005F936F937F938F939F93AF93BF93CF93F7
:10497000DF93EF93FF93C091E900CF708091EC003B
:10498000D82FD17080FDD0E81092E9008091F0001E
:10499000877F8093F00078940E94DB211092E900D9
:1049A0008091F00088608093F000CD2BCF70C09391
:1049B000E900FF91EF91DF91CF91BF91AF919F916E
:1049C0008F917F916F915F914F913F912F910F90B8
:1049D0000FBE0F901F901895E8EDF0E080818E7F5C
:1049E00080831092E2001092DA001092E100A0EEB3
:1049F000B0E08C9181608C9380818F77808319BC2B
:104A0000A7EDB0E08C918E7F8C9380818F7E808328
:104A100010927C040895CF92DF92EF92FF920F9351
:104A20001F93CF93DF93C8EDD0E088818F7E88837A
:104A3000E7EDF0E080818160808384E082BF81E0E7
:104A400080937C0488818E7F888302EE10E0F801D9
:104A500010821092DA0081EEC82ED12CF60110825D
:104A600088818F77888388818068888388818F7D1B
:104A7000888319BC1092A1041092A2041092A00481
:104A800010929F0490EEE92EF12CF70180818B7F2C
:104A9000808388818160888342E060E080E00E94BA
:104AA000F91DF60180818E7F8083F801808181600D
:104AB0008083808188608083F70180818E7F8083FE
:104AC000888180618883DF91CF911F910F91FF9042
:104AD000EF90DF90CF9008951F920F920FB60F9234
:104AE00011242F933F934F935F936F937F938F93F3
:104AF0009F93AF93BF93EF93FF938091E10082FF69
:104B000009C08091E20082FF05C08091E1008B7FA7
:104B10008093E1008091DA0080FF2AC08091D80064
:104B200080FF26C08091DA008E7F8093DA0080912A
:104B3000D90080FF18C080E189BD82E189BD09B438
:104B400000FEFDCF81E08093A10480917C0481115F
:104B50000FC00E94EC240E940B258091E20084602B
:104B60008093E20005C019BC1092A10410927C044D
:104B70008091E10080FF17C08091E20080FF13C0A8
:104B80008091E2008E7F8093E2008091E20080615C
:104B90008093E2008091D80080628093D80019BC95
:104BA00085E08093A1048091E10084FF30C0809172
:104BB000E20084FF2CC080E189BD82E189BD09B497
:104BC00000FEFDCF8091D8008F7D8093D80080912A
:104BD000E1008F7E8093E1008091E2008F7E8093E0
:104BE000E2008091E20081608093E2008091A20463
:104BF000882311F084E007C08091E30087FD02C0A4
:104C000081E001C083E08093A1048091A1048091A0
:104C1000E10083FF27C08091E20083FF23C08091E1
:104C2000E100877F8093E10082E08093A1041092ED
:104C3000A2048091E1008E7F8093E1008091E200E8
:104C40008E7F8093E2008091E20080618093E20099
:104C500042E060E080E00E94F91D8091F0008860F1
:104C60008093F000FF91EF91BF91AF919F918F9151
:104C70007F916F915F914F913F912F910F900FBE58
:104C80000F901F90189580914F07811110924F0738
:104C90000895809590914E07892380934E0708953B
:104CA00090914E0780914D07982B9093B606809176
:104CB0004F078823D9F0892B8093B60680914B014A
:104CC000882331F08091770487FF02C08EE101C014
:104CD00086E0E8EBF6E090E0815028F02191222375
:104CE000D9F39F5FF9CF91110E94432640E250E033
:104CF0006DE277E086EB96E00E94AA32892B21F1E3
:104D000080E2E6EBF6E0ADE2B7E001900D928A9525
:104D1000E1F7E0916E04F0916F043097A9F0809173
:104D20004B01882359F08091770487FF07C0809159
:104D3000B6068093B70686E08093B6060280F381BC
:104D4000E02D86EB96E00994089580E090E00E94C3
:104D5000861F80E090E00E94701F10924D070E9415
:104D60005026E7E5F7E086E0DF011D928A95E9F736
:104D70001092510710925007109252070C94E62D92
:104D800080912B079091FA06891719F08F5F877031
:104D9000FBCF08950F931F93CF93DF938091F90674
:104DA00082958F7009F05DC08091F606882309F422
:104DB00058C080912B071091FA066091F40670910B
:104DC000F506C091F706D091F80691E06F3F09F023
:104DD00090E0292F06E0811709F443C0209721F0C5
:104DE0007F3F21F030E003C031E001C0322F90E07E
:104DF00030FD34C0089FF001099FF00D1124DF0140
:104E0000A550B94F11963C911197371327C03C918B
:104E1000361324C012963C91129731111FC013967D
:104E20004D915C9114974C1B5D0B483C5105B0F4BF
:104E30008091F9068F7080618093F906E050F94FF8
:104E400080818F708061808384EF96E00E9461078B
:104E5000DF91CF911F910F910C94C026019687701E
:104E6000BACFDF91CF911F910F9108958F929F92AA
:104E7000AF92BF92DF92EF92FF920F931F93CF9367
:104E8000DF938090300290903102A0903202B09077
:104E900033024091710250917202609173027091DD
:104EA0007402842A952AA62AB72ACFE1D0E026E008
:104EB000929F7001112490E3D92E082F10E0D501A4
:104EC000C4010C2E04C0B695A795979587950A94B2
:104ED000D2F780FD04C0219790F780E014C0DC9EDB
:104EE000F001DD9EF00D1124EE0DFF1DE00FF11F0E
:104EF000EE0FFF1FE75CF64F859194910E94A71576
:104F0000019749F38C2FDF91CF911F910F91FF9063
:104F1000EF90DF90BF90AF909F908F900895CF93C8
:104F2000DF93EC010E94362720E3829FC001112409
:104F3000FC0126E0D29FE00DF11D1124EC0FF11DC4
:104F4000EE0FFF1FE75CF64F859194910E94A71525
:104F5000DF91CF910895FC01808191810E948F277C
:104F600092959F70963079F010F4925001C09A504B
:104F7000923068F4803F69F018F4883E40F409C02C
:104F8000843F29F406C0883E20F0813F11F080E084
:104F9000089581E008959F92AF92BF92CF92DF92E1
:104FA000EF92FF920F931F93CF93DF93CDB7DEB7AE
:104FB00061970FB6F894DEBF0FBECDBF8C0185E0C0
:104FC000F801DE011D9601900D928A95E1F7F80136
:104FD000E2809091F4066091F5064091F7065091B9
:104FE000F8064115510531F06F3F31F481E09F3FE4
:104FF00019F403C081E001C080E0F82FF1709F2E0A
:1050000080FD1AC1F80130812181C380D48084EFF2
:10501000A82E86E0B82EF090F606F601E41BF50BFC
:10502000FF2009F4C6C08091F906E83CF10508F0BC
:1050300091C0482F407F09F050C0621311C09313F4
:105040000FC0FE2CE1100CC08F7080618093F906B8
:10505000C5010E9461078091F906F801858329C185
:10506000CD2831F02F3F31F481E03F3F19F403C0E8
:1050700081E001C080E080FD03C081E08E2502C098
:1050800080E090E0F82FF170FF2E80FF1CC080912F
:105090002B074091FA0656E0841709F4E8C090E027
:1050A000589FF001599FF00D1124E550F94F61818F
:1050B000261306C06081631303C06281E61203C039
:1050C00001968770E9CFFE2CEE2009F4F2C08091A2
:1050D000F90681608093F90649C0621306C09313F4
:1050E00004C0E11002C0F80186C0C8010E94AB27CD
:1050F000882351F1EE2041F12091F906822F82950B
:105100008F7090E0029774F08091F4069091F5060C
:1051100098878F831986DB86CA862C87CE010796EF
:105120000E94610786E0F801A4EFB6E001900D92BD
:105130008A95E1F70E94CA260AC06217C9F0C80121
:105140000E94AB2781111EC0C8010E946107FF2485
:10515000F394AFC0482F407F81F784EF96E00E9420
:10516000610786E0F50111928A95E9F7F12CA1C05B
:105170009313E5CFE110E3CFF8018583C8010E94C6
:10518000610754C0EE2001F32091F906822F829529
:105190008F7090E0029734F28091F4069091F506BA
:1051A0009A8389831B82DD82CC822E83CE01019675
:1051B000B7CFE83CF105D0F5FE2CEE2029F26213C2
:1051C00027C0931325C02091F90620FD18C0822F17
:1051D00082958F70482F50E04115510581F0F801FC
:1051E00025834F30510541F08F5F982F9295907F26
:1051F000822F8F70892B8583C8010E94610786E00A
:10520000F801A4EFB6E001900D928A95E1F751C044
:10521000C8010E94AB27811185CF8091F90681607A
:105220008093F906C8010E94610743C086E0F5013A
:1052300011928A95E9F73DC0EE2009F485CFC801A7
:105240000E94AB27F82E882309F47ECF86E0F80170
:10525000A4EFB6E001900D928A95E1F78091F406F3
:105260009091F5060E948F270E94CA2622C03D8792
:105270002E878D859E850E948F27292F22952F703E
:10528000223028F49F7039F0811105C00BC0243002
:1052900028F49F7049F4805E883020F0C8010E9495
:1052A00061079F2CF92C05C0F8019581907F99F733
:1052B000F9CF8F2D61960FB6F894DEBF0FBECDBF2C
:1052C000DF91CF911F910F91FF90EF90DF90CF90E2
:1052D000BF90AF909F900895292F220F920F990FA2
:1052E000890F682F669566956695982F977085E06B
:1052F000689FB001112440E050E080E0FB01E40F22
:10530000F51FEA52F94F208130E0092E02C0369590
:1053100027950A94E2F721703327042E01C0220F4B
:105320000A94EAF7822B4F5F5F4F4530510531F702
:105330000895292F220F920F990F890FE82FE695D4
:10534000E695E695877051E001C0550F8A95EAF71A
:1053500085E0E89FF0011124EA52F94F20E030E0A7
:1053600070E04081CB01022E02C0969587950A9489
:10537000E2F78170819584278523842781932F5FAD
:105380003F4F2530310569F70895609330027093DF
:10539000310280933202909333020C94A5260F932E
:1053A0001F9341E050E060E070E004C0440F551FDF
:1053B000661F771F8A95D2F7409550956095709536
:1053C0008091300290913102A0913202B09133026B
:1053D0008A019B01082319232A233B23C901B80111
:1053E0001F910F910C94C52920912C078095822341
:1053F00080932C07982F977099F430E0482F082E4F
:10540000000C550B2417350759F09091780492FD44
:1054100007C08595859585950E94CF2910922C0708
:105420000895CF93C0917804C2FB992790F99817FB
:1054300099F080FBC2F9C09378046091770484E00E
:1054400090E00E94C3316C2F82E290E00E94C33151
:1054500082E0CF910C94F429CF9108950F931F937C
:1054600041E050E060E070E004C0440F551F661F4B
:10547000771F8A95D2F78091300290913102A091E6
:105480003202B09133028A019B01082B192B2A2B7F
:105490003B2BC901B8011F910F910C94C529609352
:1054A00071027093720280937302909374020C9451
:1054B000A52610924E0780914B01882331F08091F0
:1054C000770487FF02C08EE101C086E0E8EBF6E0DA
:1054D000DF011D928A95E9F70C94A52630914701CA
:1054E00080915E0480FF16C0E091460163E0E69F74
:1054F000F0011124E255FD4F539A8BB1877F9BB188
:1055000098602FB7F894AF0163E0369F400D511DAE
:10551000112414C08091480190914901891720F706
:10552000E82FF0E0AF01440F551FE40FF51FE255DF
:10553000FD4F1182108212828F5FF0CFE417F507C2
:1055400089F0319168E09BB9000000C037FF8BB94A
:10555000330F000000C000C000C08BB900C06A95C6
:1055600091F7ECCF2FBF8FE594E00197F1F700C0E2
:105570000000089590915E0490FF16C0909148013C
:1055800020914901921770F4E92FF0E0DF01AA0F92
:10559000BB1FEA0FFB1FE255FD4F818360834283EF
:1055A0009F5FF0CF0C946E2A089580915E04282F9F
:1055B000269530E02115310519F48170826005C00F
:1055C0002B32310524F08170846580935E048091D4
:1055D0006104893718F088E7809361040895CF92B9
:1055E000DF92EF92FF926B017C010E94D52AB701F6
:1055F000A60188E090E0FF90EF90DF90CF900C94B0
:10560000D53180916204882319F08150809362041F
:1056100060915E0470915F048091600490916104D8
:105620000C94EF2A80916204833018F48F5F80938A
:10563000620460915E0470915F04809160049091B7
:1056400061040C94EF2AEEE5F4E083E0808311829C
:105650008FEF828388E783831482A8EAB2E01296F0
:105660008C911297836012968C93608171818281F4
:1056700093810C94EF2AAF92BF92CF92DF92EF9278
:10568000FF920F931F93CF93DF93E82EF62EE9013D
:10569000493708F048E7E42FF0E0F11006C0E7547E
:1056A000F54FE4914E2F2E2F71C00F2D10E0E754CF
:1056B000F54F4491F42FC42ED12C26E0E29EC00178
:1056C00011242FEF30E0B9010E9436315BEA560316
:1056D000C001579F900D11248E0D911D8E0D911DAF
:1056E000582F550F580FD901A01BB10BAC9DC0010D
:1056F000AD9D900DBC9D900D1124E92FF59ED0011C
:105700001124AB2FBB277901EA1AFB0AEC9CD001CC
:10571000ED9CB00DFC9CB00D11245901A51AB108E7
:10572000A09E7001A19EF00CB09EF00C1124EF2CF5
:10573000FF242E193F092C9D80012D9D100D3C9DAD
:10574000100D1124212F6230710591F048F461157C
:105750007105E1F061307105B9F4242F4B2F16C0AB
:105760006430710569F040F06630710579F00CC065
:10577000242F492FE12F0AC0492FEF2F2B2F06C0CE
:10578000292FE42F412F02C0292FEB2F4983288393
:10579000EA83DF91CF911F910F91FF90EF90DF90FF
:1057A000CF90BF90AF900895AF92BF92CF92DF920B
:1057B000EF92FF920F931F93CF93DF9300D01F922E
:1057C000CDB7DEB7182FF62E042FE22E90915E048F
:1057D00090FF7EC0E92FE695AE2FB0E0A252BE4FFB
:1057E0008C918093A8029E7F923061F49E012F5F7E
:1057F0003F4F812F0E943B2B4B8169818A810E9400
:10580000BA2A43C0823019F4009161043EC0863048
:1058100019F410915F0439C08930D9F38931A9F5A1
:10582000E9518E2F8170D82EE695F0E0E754F44FC1
:10583000A590B490C12CBB2460914A01C61618F5FE
:105840002C2D30E0A29EC001A39E900DB29E900D23
:10585000112470E00E943631812FD11002C0860FD2
:1058600001C0861B90914801290F311DA901440FE9
:10587000551F240F351F22553D4F402F6F2D0E947D
:105880003B2BC394D9CF0E946E2A80915F041813DA
:1058900008C080916004F81204C080916104081768
:1058A00029F08091AA0282608093AA0210935F047B
:1058B000F092600400936104EE2051F060915E0468
:1058C00070915F0480916004909161040E94EF2ABE
:1058D0000F900F900F90DF91CF911F910F91FF903C
:1058E000EF90DF90CF90BF90AF900895EEE5F4E099
:1058F000438121E1421B08F440E021E06281818183
:105900000C94D42BEEE5F4E0438121E1420F08F43E
:105910004FEF21E0628181810C94D42BEEE5F4E01D
:10592000628121E1621B08F460E021E04381818112
:105930000C94D42BEEE5F4E0628121E1620F08F4CF
:105940006FEF21E0438181810C94D42BEEE5F4E0EC
:10595000818121E0438162818A500C94D42BEEE551
:10596000F4E0818121E043816281865F0C94D42B35
:10597000CF93DF9300D01F92CDB7DEB790915E0436
:1059800090FF0AC09E012F5F3F4F0E943B2B4B812F
:1059900069818A810E94BA2A0F900F900F90DF913F
:1059A000CF9108958D3E39F490915A0797FF35C0F5
:1059B00010925A0759C08E3E29F490915A07191631
:1059C000BCF32BC0909159078F3E29F497FF25C057
:1059D0001092590749C0803F19F41916CCF31DC025
:1059E00090915B07893F29F41916BCF410925B076C
:1059F0003BC08A3F19F497FF10C0F8CF8B3F39F4B2
:105A000090915C0797FF09C010925C072DC08C3FF6
:105A100021F490915C071916BCF39FE0980F983021
:105A200080F421E030E0A90102C0440F551F9A958F
:105A3000E2F7CA018095909158078923809358070F
:105A400013C08D3F21F4809152078E7F0BC08E3F93
:105A500021F4809152078D7F05C08F3F29F48091FA
:105A600052078B7F8093520780915907811106C09E
:105A700080915A07811102C01092510780915B07F3
:105A8000811106C080915C07811102C010925007FD
:105A900008958091520780FD16C081FD16C082FDD9
:105AA00018C080915007882391F0883290F428E044
:105AB000829FC001112468E270E00E947432862F38
:105AC000672B29F007C082E0089584E0089581E003
:105AD000089588E008958091520780FD14C081FDEB
:105AE00014C082FD16C080915107882381F08E3149
:105AF00080F420E5829FC00111246EE170E00E94D5
:105B00007432862F089584E1089588E2089588E02C
:105B1000089580E508958D3E21F40E946B2D8195B6
:105B200004C08E3E29F40E946B2D80935A0708957D
:105B30008F3E21F40E946B2D819504C0803F29F493
:105B40000E946B2D809359070895893F19F40E9494
:105B5000492D05C08A3F31F40E94492D81958093DB
:105B60005B0708958B3F21F40E94492D819504C065
:105B70008C3F29F40E94492D80935C0708959FE093
:105B8000980F983078F421E030E0A90102C0440F6A
:105B9000551F9A95E2F7CA0190915807892B809377
:105BA000580708958D3F21F48091520781600BC002
:105BB0008E3F21F480915207826005C08F3F29F407
:105BC0008091520784608093520708950E94DE1EE0
:105BD00020915907211104C020915A07222321F056
:105BE000909356078093550720915B07211104C0BD
:105BF00020915C07222321F0909354078093530750
:105C0000E0916E04F0916F04309749F082E0809348
:105C100057070480F581E02D87E597E00994089502
:105C200090915E0490FF3BC09170811102C0926020
:105C300006C08B3210F0946502C0880F982B9093A9
:105C40005E048091AA0281608093AA02662351F0CB
:105C500060915E0470915F04809160049091610492
:105C60000E94EF2A60915E04669570E04BE050E080
:105C700088E391E00E949D32892B19F00E94BF2099
:105C800002C00E94C62081E08093A50220E04091DE
:105C900061046091600480915F040C94D42B08959A
:105CA00080915E048695815009F48AE261E00C944B
:105CB000102E80915E0486958F5F8B3208F081E014
:105CC00061E00C94102E1092B9008CE08093B80023
:105CD00008959F92AF92BF92CF92DF92EF92FF9280
:105CE0000F931F93CF93DF93B82EEB010E94DE1E1C
:105CF0006C01C431D10558F0CF3F8FEFD80759F070
:105D0000CE0164E170E00E9436317B0107C0EE24D1
:105D1000E394F12C03C025E0E22EF12C84E8A82EB8
:105D200094EA992E1092BC009092BC000E94DE1E54
:105D30008C018091BC0087FD08C00E94DE1E801B84
:105D4000910B8E159F05A8F32AC08091B900887F1A
:105D5000883041F08091B900887F803119F00FEFD1
:105D60001FEF1FC0B092BB00A092BC000E94DE1EBD
:105D70008C018091BC0087FD08C00E94DE1E801B44
:105D8000910B8E159F05A8F30AC08091B900887FFA
:105D9000883111F0803419F700E010E00EC00EEFEA
:105DA0001FEFCF3F8FEFD80709F4BCCFC6010E9489
:105DB000C31E8C179D0708F4B5CFC801DF91CF91A2
:105DC0001F910F91FF90EF90DF90CF90BF90AF9019
:105DD0009F9008950F931F93CF93DF93EB018093D0
:105DE000BB0084E88093BC000E94DE1E8C01809181
:105DF000BC0087FD0EC0CF3F8FEFD807C1F30E94D4
:105E0000DE1E801B910B8C179D0788F38EEF9FEF92
:105E10000CC02091B900287F81E090E0283211F475
:105E200080E090E0919581959109DF91CF911F914C
:105E30000F910895CF92DF92EF92FF920F931F93ED
:105E4000CF93DF936B018A017901B9010E94692E1A
:105E5000E6010C0D1D1DC017D10761F424E9209344
:105E6000BC00DF91CF911F910F91FF90EF90DF90D9
:105E7000CF90089597FDF2CFB70189910E94EA2E45
:105E8000EACFCF92DF92EF92FF920F931F93CF93BF
:105E9000DF93C62F6A017901B8010E94692E97FD30
:105EA00011C0B8018C2F0E94EA2EE601EC0CFD1CFB
:105EB000CE15DF0539F097FD05C0B80189910E9424
:105EC000EA2EF6CF24E92093BC00DF91CF911F91F9
:105ED0000F91FF90EF90DF90CF90089584E9809329
:105EE000BC0008958EE14A9B02C08150E1F74A9BB5
:105EF000FECF08955A9880E28A95F1F75A9A08954C
:105F0000FC012AE02A95F1F728E090E080E031E0FA
:105F100040E14A95F1F7880F4A9B02C081609327C0
:105F200000C0000040E14A95F1F7215089F720E1D7
:105F30002A95F1F729B100C0000030E13A95F1F758
:105F400022FB222720F992272081920F9083089527
:105F5000EF92FF920F931F93CF93DF931F92CDB7D2
:105F6000DEB719828C017C01E60EF11C0E151F05AF
:105F700051F00E94722FCE0101960E94802FF801ED
:105F800081938F01F3CF81E09981911180E00F908F
:105F9000DF91CF911F910F91FF90EF900895529A4A
:105FA0005A9A089552985A9AEA9AE9E6F0E080815E
:105FB0008F7C80830895615091E001C0990F6A95AC
:105FC000EAF720E031E0992361F0492F482319F0E6
:105FD0005A9A232701C05A9840E24A95F1F79695BC
:105FE000F2CF222311F05A9A01C05A9880E28A9582
:105FF000F1F75A980895FF920F931F93CF93DF9371
:10600000EC018C01060F111DC017D10741F0F9906A
:106010000E947A2F68E08F2D0E94DB2FF5CFDF9151
:10602000CF911F910F91FF9008951F920F920FB67D
:106030000F9211240F931F932F933F934F935F93CE
:106040006F937F938F939F93AF93BF93EF93FF9340
:10605000CF93DF931F92CDB7DEB719820E94722FC4
:10606000CE0101960E94802F082F06950695069571
:10607000902F96959570202F2570920F292F2370C1
:1060800096959695920F877089135FC089818111CB
:106090005CC0053008F059C080E18A95F1F75A9A42
:1060A000529A82E08A95F1F700C05A9888E0089FDA
:1060B00080011124D801A85EBE4F1696ED91FC9187
:1060C00017973097A9F06091DC017091DD0114966B
:1060D0002D913C911597260F371F11968D919C910C
:1060E0001297680F791F13964C9113978C9109950D
:1060F000F801E85EFE4F6381662351F08091DC0178
:106100009091DD0124813581820F931F0E94FB2F26
:106110000E947A2F80E18A95F1F75A9852985A9AFC
:1061200080E18A95F1F7F801E85EFE4F6081662311
:1061300051F08091DC019091DD0121813281820F4B
:10614000931F0E94A82F0E94722F0F90DF91CF9172
:10615000FF91EF91BF91AF919F918F917F916F913F
:106160005F914F913F912F911F910F910F900FBE13
:106170000F901F9018950F931F93CF93DF93853047
:1061800091050CF06DC0EC01F894529A5A9885E094
:106190008A95F1F700009C2F969595702C2F25700D
:1061A000920F892F83709695969523E0CC0FDD1F73
:1061B0002A95E1F7980F8E01092B0E947A2F84E02F
:1061C0008A95F1F700C068E0802F0E94DB2F80E104
:1061D0008A95F1F752985A9A4A9902C000C0FCCFAA
:1061E00087E090E04A9B08C0019721F4529A5A9A9E
:1061F000789436C000C0F6CFFE01E85EFE4F6381A2
:10620000662381F08091DC019091DD01248135814C
:10621000820F931F0E94A82F811104C0529A5A9A8C
:1062200078941FC00E94722F80E28A95F1F75A98E5
:10623000529A80E18A95F1F7C85EDE4F6881662345
:1062400051F08091DC019091DD0129813A81820F2A
:10625000931F0E94FB2F0E947A2F789481E001C047
:1062600080E0DF91CF911F910F910895AA1BBB1B76
:1062700051E107C0AA1FBB1FA617B70710F0A61B46
:10628000B70B881F991F5A95A9F780959095BC0167
:10629000CD0108958F929F92AF92BF92CF92DF92DD
:1062A000EF92FF92CF93DF93EC01688179818A812D
:1062B0009B81611571058105910521F464E279EDF9
:1062C0008BE597E02DE133EF41E050E00E94F7319C
:1062D00049015A019B01AC01A7EAB1E40E941632C0
:1062E0006B017C01ACEEB4EFA50194010E94243255
:1062F000DC01CB018C0D9D1DAE1DBF1DB7FF03C082
:106300000197A109B04888839983AA83BB839F77AB
:10631000DF91CF91FF90EF90DF90CF90BF90AF9043
:106320009F908F9008950E944A31089580E091E0F7
:106330000E944A310895A0E0B0E08093000190935C
:106340000101A0930201B09303010895FB01DC0158
:1063500002C005900D9241505040D8F70895F99928
:10636000FECF92BD81BDF89A992780B50895A6E128
:10637000B0E044E050E00C94E931A8E1B0E042E044
:1063800050E00C94E931262FF999FECF92BD81BDE2
:10639000F89A019700B4021639F01FBA20BD0FB663
:1063A000F894FA9AF99A0FBE08950396272F0E943F
:1063B000C4310E94C331252F0E94C431242F0C9474
:1063C000C4310196272F0E94C4310C94C331DC01E3
:1063D000CB01FC01F999FECF06C0F2BDE1BDF89AF0
:1063E000319600B40D9241505040B8F70895052EF3
:1063F00097FB1EF400940E940E3257FD07D00E94B6
:10640000293207FC03D04EF40C940E32509540957F
:10641000309521953F4F4F4F5F4F08959095809550
:10642000709561957F4F8F4F9F4F08950E944B321B
:10643000A59F900DB49F900DA49F800D911D1124D8
:106440000895B7FF0C9416320E941632821B930BEC
:106450000895A1E21A2EAA1BBB1BFD010DC0AA1FA5
:10646000BB1FEE1FFF1FA217B307E407F50720F0BD
:10647000A21BB30BE40BF50B661F771F881F991F38
:106480001A9469F760957095809590959B01AC0181
:10649000BD01CF010895A29FB001B39FC001A39F8A
:1064A000700D811D1124911DB29F700D811D11244D
:1064B000911D0895991B79E004C0991F961708F063
:1064C000961B881F7A95C9F78095089587FB082E3B
:1064D000062687FD819567FD61950E945A320EF46C
:1064E000919507FC8195089597FB072E16F400946B
:1064F00007D077FD09D00E94363107FC05D03EF465
:10650000909581959F4F0895709561957F4F08955F
:10651000EE0FFF1F0590F491E02D09940E944B327D
:10652000332312F48A1B9B0B0C9498320E944B323B
:10653000B7FF0895821B930B0895FC014150504012
:1065400030F001900616D1F73197CF0108958827D2
:1065500099270895FB01DC0104C08D9101908019F9
:1065600021F441505040C8F7881B990B0895FB0156
:10657000DC0102C001900D9241505040D8F70895BF
:10658000AEE0B0E0E6ECF2E30C948F350D891E89A5
:106590008F89988D26E02C831A83098397FF02C088
:1065A00080E090E801979E838D83AE01455E5F4F4A
:1065B000698D7A8DCE0101960E94F0324D815E8107
:1065C00057FD0AC02F813885421753070CF49A01F2
:1065D000F801E20FF31F10822E96E4E00C94AB3525
:1065E000ABE0B0E0E6EFF2E30C9481356C017B01A7
:1065F0008A01FC0117821682838181FFCCC1CE0102
:1066000001963C01F6019381F70193FD859193FF7B
:1066100081917F01882309F4BAC1853239F493FD51
:10662000859193FF81917F01853229F4B60190E035
:106630000E94E734E7CF912C212C312CFFE1F31598
:10664000D8F08B3279F038F4803279F08332A1F4CB
:10665000232D20611DC08D3261F0803369F4232D1C
:10666000216016C0832D8260382EE32DE4603E2E1B
:106670002AC0F32DF8601DC037FC2DC020ED280F77
:106680002A3040F08E32B9F436FC81C1232D2064CB
:10669000322E19C036FE06C08AE0989E200D1124C5
:1066A000922E11C0EAE02E9E200D1124222EF32DF1
:1066B000F0623F2E08C08C3621F4832D8068382E7E
:1066C00002C0883641F4F70193FD859193FF8191D3
:1066D0007F018111B3CF982F9F7D9554933028F47B
:1066E0000C5F1F4F9FE399830DC0833631F08337D2
:1066F00071F0833509F059C021C0F8018081898388
:106700000E5F1F4F88248394912C530113C02801DE
:10671000F2E04F0E511CF801A080B18036FE03C09C
:10672000692D70E002C06FEF7FEFC5010E94DC347D
:106730004C018201F32DFF773F2E16C0280122E085
:10674000420E511CF801A080B18036FE03C0692DB5
:1067500070E002C06FEF7FEFC5010E94D1344C01A1
:10676000F32DF0683F2E820133FC1BC0822D90E098
:1067700088169906B0F4B60180E290E00E94E734F2
:106780002A94F4CFF50137FC859137FE81915F01A2
:10679000B60190E00E94E73421102A9421E0821A89
:1067A00091088114910471F7E8C0843611F089369C
:1067B00041F5F80137FE07C06081718182819381C4
:1067C0000C5F1F4F08C060817181072E000C880B81
:1067D000990B0E5F1F4FF32DFF763F2E97FF09C0D9
:1067E00090958095709561957F4F8F4F9F4FF06882
:1067F0003F2E2AE030E0A3010E942335882E861820
:1068000045C0853731F4232D2F7EB22E2AE030E0AB
:1068100025C0932D997FB92E8F36C1F018F4883595
:1068200079F0B5C0803719F0883721F0B0C0E92F72
:10683000E061BE2EB4FE0DC0FB2DF460BF2E09C07A
:1068400034FE0AC0292F2660B22E06C028E030E0B0
:1068500005C020E130E002C020E132E0F801B7FEDF
:1068600007C060817181828193810C5F1F4F06C0D8
:106870006081718180E090E00E5F1F4FA3010E9454
:106880002335882E8618FB2DFF773F2E36FE0DC050
:10689000232D2E7FA22E891458F434FE0BC032FC17
:1068A00009C0832D8E7EA82E05C0B82CA32C03C052
:1068B000B82C01C0B92CA4FE0FC0FE01E80DF11DDB
:1068C0008081803321F49A2D997EA92E09C0A2FEE1
:1068D00006C0B394B39404C08A2D867809F0B394AB
:1068E000A3FC11C0A0FE06C0B21488F4280C922CA0
:1068F0009B180EC0B21460F4B60180E290E00E94D2
:10690000E734B394F7CFB21418F42B1802C0982CC4
:10691000212CA4FE10C0B60180E390E00E94E73471
:10692000A2FE17C0A1FC03C088E790E002C088E582
:1069300090E0B6010CC08A2D867859F0A1FE02C005
:106940008BE201C080E2A7FC8DE2B60190E00E94DC
:10695000E734891438F4B60180E390E00E94E7340C
:106960009A94F7CF8A94F301E80DF11D8081B60166
:1069700090E00E94E7348110F5CF222009F442CE46
:10698000B60180E290E00E94E7342A94F6CFF60147
:106990008681978102C08FEF9FEF2B96E2E10C94E6
:1069A0009D35FC010590615070400110D8F780952D
:1069B00090958E0F9F1F0895FC01615070400190CB
:1069C0000110D8F7809590958E0F9F1F08950F9313
:1069D0001F93CF93DF93FB01238121FD03C08FEF32
:1069E0009FEF2CC022FF16C046815781248135813C
:1069F0004217530744F4A081B1819D012F5F3F4F9F
:106A0000318320838C93268137812F5F3F4F3783DB
:106A1000268314C08B01EC01FB010084F185E02D7D
:106A20000995892BE1F6D80116968D919C911797BF
:106A3000019617969C938E931697CE01DF91CF9176
:106A40001F910F910895FA01AA27283051F12031A2
:106A500081F1E8946F936E7F6E5F7F4F8F4F9F4FF2
:106A6000AF4FB1E03ED0B4E03CD0670F781F891F34
:106A70009A1FA11D680F791F8A1F911DA11D6A0F02
:106A8000711D811D911DA11D20D009F468943F91B5
:106A90002AE0269F11243019305D3193DEF6CF01B4
:106AA0000895462F4770405D4193B3E00FD0C9F77A
:106AB000F6CF462F4F70405D4A3318F0495D31FDE7
:106AC0004052419302D0A9F7EACFB4E0A69597953A
:106AD000879577956795BA95C9F700976105710510
:106AE00008959B01AC010A2E06945795479537955A
:106AF0002795BA95C9F7620F731F841F951FA01DB4
:106B000008952F923F924F925F926F927F928F9251
:106B10009F92AF92BF92CF92DF92EF92FF920F932C
:106B20001F93CF93DF93CDB7DEB7CA1BDB0B0FB636
:106B3000F894DEBF0FBECDBF09942A8839884888F3
:106B40005F846E847D848C849B84AA84B984C88489
:106B5000DF80EE80FD800C811B81AA81B981CE0F80
:106B6000D11D0FB6F894DEBF0FBECDBFED01089565
:046B7000F894FFCFC7
:106B74000100000001A619FC19DD19D919D519A5C0
:106B8400190021007F220003000000010000000022
:106B940000000004010000000405000000000000E3
:106BA400080900000000000001191A1B1C1D1E1F0B
:106BB40020212201020100360036360125647825A1
:106BC400642C206B253264203A2025630020202089
:106BD400206162636465666768696A6B6C6D6E6F79
:106BE400707172737475767778797A31323334359B
:106BF4003637383930524542545F2D3D5B5D5C2356
:106C04003B27602C2E2F202020946697C6F4F5F69F
:106C1400F731330008101818100800818283E2004D
:106C2400E900EA00B500B600B700CD008301CC004E
:106C34008A019201940121022302240225022602E0
:106C440027022A02B300B4006F0070008C02000116
:106C5400020202020606060909090909090F0F0FB3
:106C64000F0F0F15151518191919191919191919BB
:0A6C740019232425252525252500D8
:00000001FF
